Archive member included to satisfy reference by file (symbol)

/usr/lib/gcc/arm-none-eabi/10.2.0/../../../../arm-none-eabi/lib/thumb/v7e-m/nofp/libc_nano.a(lib_a-atexit.o)
                              /usr/lib/gcc/arm-none-eabi/10.2.0/../../../../arm-none-eabi/lib/thumb/v7e-m/nofp/crt0.o (atexit)
/usr/lib/gcc/arm-none-eabi/10.2.0/../../../../arm-none-eabi/lib/thumb/v7e-m/nofp/libc_nano.a(lib_a-exit.o)
                              /usr/lib/gcc/arm-none-eabi/10.2.0/../../../../arm-none-eabi/lib/thumb/v7e-m/nofp/crt0.o (exit)
/usr/lib/gcc/arm-none-eabi/10.2.0/../../../../arm-none-eabi/lib/thumb/v7e-m/nofp/libc_nano.a(lib_a-fini.o)
                              /usr/lib/gcc/arm-none-eabi/10.2.0/../../../../arm-none-eabi/lib/thumb/v7e-m/nofp/crt0.o (__libc_fini_array)
/usr/lib/gcc/arm-none-eabi/10.2.0/../../../../arm-none-eabi/lib/thumb/v7e-m/nofp/libc_nano.a(lib_a-impure.o)
                              /usr/lib/gcc/arm-none-eabi/10.2.0/../../../../arm-none-eabi/lib/thumb/v7e-m/nofp/libc_nano.a(lib_a-exit.o) (_global_impure_ptr)
/usr/lib/gcc/arm-none-eabi/10.2.0/../../../../arm-none-eabi/lib/thumb/v7e-m/nofp/libc_nano.a(lib_a-init.o)
                              /usr/lib/gcc/arm-none-eabi/10.2.0/../../../../arm-none-eabi/lib/thumb/v7e-m/nofp/crt0.o (__libc_init_array)
/usr/lib/gcc/arm-none-eabi/10.2.0/../../../../arm-none-eabi/lib/thumb/v7e-m/nofp/libc_nano.a(lib_a-memcpy-stub.o)
                              ESF/mcu/src/startup_same54.o (memcpy)
/usr/lib/gcc/arm-none-eabi/10.2.0/../../../../arm-none-eabi/lib/thumb/v7e-m/nofp/libc_nano.a(lib_a-memset.o)
                              /usr/lib/gcc/arm-none-eabi/10.2.0/../../../../arm-none-eabi/lib/thumb/v7e-m/nofp/crt0.o (memset)
/usr/lib/gcc/arm-none-eabi/10.2.0/../../../../arm-none-eabi/lib/thumb/v7e-m/nofp/libc_nano.a(lib_a-__atexit.o)
                              /usr/lib/gcc/arm-none-eabi/10.2.0/../../../../arm-none-eabi/lib/thumb/v7e-m/nofp/libc_nano.a(lib_a-atexit.o) (__register_exitproc)
/usr/lib/gcc/arm-none-eabi/10.2.0/../../../../arm-none-eabi/lib/thumb/v7e-m/nofp/libc_nano.a(lib_a-__call_atexit.o)
                              /usr/lib/gcc/arm-none-eabi/10.2.0/../../../../arm-none-eabi/lib/thumb/v7e-m/nofp/libc_nano.a(lib_a-__atexit.o) (__call_exitprocs)
/usr/lib/gcc/arm-none-eabi/10.2.0/../../../../arm-none-eabi/lib/thumb/v7e-m/nofp/libc_nano.a(lib_a-lock.o)
                              /usr/lib/gcc/arm-none-eabi/10.2.0/../../../../arm-none-eabi/lib/thumb/v7e-m/nofp/libc_nano.a(lib_a-__atexit.o) (__retarget_lock_acquire_recursive)

Allocating common symbols
Common symbol       size              file

__lock___atexit_recursive_mutex
                    0x1               /usr/lib/gcc/arm-none-eabi/10.2.0/../../../../arm-none-eabi/lib/thumb/v7e-m/nofp/libc_nano.a(lib_a-lock.o)
__lock___arc4random_mutex
                    0x1               /usr/lib/gcc/arm-none-eabi/10.2.0/../../../../arm-none-eabi/lib/thumb/v7e-m/nofp/libc_nano.a(lib_a-lock.o)
__lock___env_recursive_mutex
                    0x1               /usr/lib/gcc/arm-none-eabi/10.2.0/../../../../arm-none-eabi/lib/thumb/v7e-m/nofp/libc_nano.a(lib_a-lock.o)
__lock___sinit_recursive_mutex
                    0x1               /usr/lib/gcc/arm-none-eabi/10.2.0/../../../../arm-none-eabi/lib/thumb/v7e-m/nofp/libc_nano.a(lib_a-lock.o)
__lock___malloc_recursive_mutex
                    0x1               /usr/lib/gcc/arm-none-eabi/10.2.0/../../../../arm-none-eabi/lib/thumb/v7e-m/nofp/libc_nano.a(lib_a-lock.o)
__lock___at_quick_exit_mutex
                    0x1               /usr/lib/gcc/arm-none-eabi/10.2.0/../../../../arm-none-eabi/lib/thumb/v7e-m/nofp/libc_nano.a(lib_a-lock.o)
__lock___dd_hash_mutex
                    0x1               /usr/lib/gcc/arm-none-eabi/10.2.0/../../../../arm-none-eabi/lib/thumb/v7e-m/nofp/libc_nano.a(lib_a-lock.o)
__lock___tz_mutex   0x1               /usr/lib/gcc/arm-none-eabi/10.2.0/../../../../arm-none-eabi/lib/thumb/v7e-m/nofp/libc_nano.a(lib_a-lock.o)
__lock___sfp_recursive_mutex
                    0x1               /usr/lib/gcc/arm-none-eabi/10.2.0/../../../../arm-none-eabi/lib/thumb/v7e-m/nofp/libc_nano.a(lib_a-lock.o)

Discarded input sections

 .text          0x0000000000000000        0x0 /usr/lib/gcc/arm-none-eabi/10.2.0/thumb/v7e-m/nofp/crti.o
 .data          0x0000000000000000        0x0 /usr/lib/gcc/arm-none-eabi/10.2.0/thumb/v7e-m/nofp/crti.o
 .bss           0x0000000000000000        0x0 /usr/lib/gcc/arm-none-eabi/10.2.0/thumb/v7e-m/nofp/crti.o
 .text          0x0000000000000000        0x0 /usr/lib/gcc/arm-none-eabi/10.2.0/thumb/v7e-m/nofp/crtbegin.o
 .data          0x0000000000000000        0x0 /usr/lib/gcc/arm-none-eabi/10.2.0/thumb/v7e-m/nofp/crtbegin.o
 .bss           0x0000000000000000        0x0 /usr/lib/gcc/arm-none-eabi/10.2.0/thumb/v7e-m/nofp/crtbegin.o
 .data.__dso_handle
                0x0000000000000000        0x4 /usr/lib/gcc/arm-none-eabi/10.2.0/thumb/v7e-m/nofp/crtbegin.o
 .text          0x0000000000000000       0x70 /usr/lib/gcc/arm-none-eabi/10.2.0/../../../../arm-none-eabi/lib/thumb/v7e-m/nofp/crt0.o
 .data          0x0000000000000000        0x0 /usr/lib/gcc/arm-none-eabi/10.2.0/../../../../arm-none-eabi/lib/thumb/v7e-m/nofp/crt0.o
 .bss           0x0000000000000000        0x0 /usr/lib/gcc/arm-none-eabi/10.2.0/../../../../arm-none-eabi/lib/thumb/v7e-m/nofp/crt0.o
 .ARM.extab     0x0000000000000000        0x0 /usr/lib/gcc/arm-none-eabi/10.2.0/../../../../arm-none-eabi/lib/thumb/v7e-m/nofp/crt0.o
 .ARM.exidx     0x0000000000000000       0x10 /usr/lib/gcc/arm-none-eabi/10.2.0/../../../../arm-none-eabi/lib/thumb/v7e-m/nofp/crt0.o
 .ARM.attributes
                0x0000000000000000       0x1c /usr/lib/gcc/arm-none-eabi/10.2.0/../../../../arm-none-eabi/lib/thumb/v7e-m/nofp/crt0.o
 .group         0x0000000000000000        0xc ESF/mcu/src/startup_same54.o
 .group         0x0000000000000000        0xc ESF/mcu/src/startup_same54.o
 .group         0x0000000000000000        0xc ESF/mcu/src/startup_same54.o
 .group         0x0000000000000000        0xc ESF/mcu/src/startup_same54.o
 .group         0x0000000000000000        0xc ESF/mcu/src/startup_same54.o
 .group         0x0000000000000000        0xc ESF/mcu/src/startup_same54.o
 .group         0x0000000000000000        0xc ESF/mcu/src/startup_same54.o
 .group         0x0000000000000000        0xc ESF/mcu/src/startup_same54.o
 .group         0x0000000000000000        0xc ESF/mcu/src/startup_same54.o
 .group         0x0000000000000000        0xc ESF/mcu/src/startup_same54.o
 .group         0x0000000000000000        0xc ESF/mcu/src/startup_same54.o
 .group         0x0000000000000000        0xc ESF/mcu/src/startup_same54.o
 .group         0x0000000000000000        0xc ESF/mcu/src/startup_same54.o
 .group         0x0000000000000000        0xc ESF/mcu/src/startup_same54.o
 .group         0x0000000000000000        0xc ESF/mcu/src/startup_same54.o
 .group         0x0000000000000000        0xc ESF/mcu/src/startup_same54.o
 .group         0x0000000000000000        0xc ESF/mcu/src/startup_same54.o
 .group         0x0000000000000000        0xc ESF/mcu/src/startup_same54.o
 .group         0x0000000000000000        0xc ESF/mcu/src/startup_same54.o
 .group         0x0000000000000000        0xc ESF/mcu/src/startup_same54.o
 .group         0x0000000000000000        0xc ESF/mcu/src/startup_same54.o
 .group         0x0000000000000000        0xc ESF/mcu/src/startup_same54.o
 .group         0x0000000000000000        0xc ESF/mcu/src/startup_same54.o
 .group         0x0000000000000000        0xc ESF/mcu/src/startup_same54.o
 .group         0x0000000000000000        0xc ESF/mcu/src/startup_same54.o
 .group         0x0000000000000000        0xc ESF/mcu/src/startup_same54.o
 .group         0x0000000000000000        0xc ESF/mcu/src/startup_same54.o
 .group         0x0000000000000000        0xc ESF/mcu/src/startup_same54.o
 .group         0x0000000000000000        0xc ESF/mcu/src/startup_same54.o
 .group         0x0000000000000000        0xc ESF/mcu/src/startup_same54.o
 .group         0x0000000000000000        0xc ESF/mcu/src/startup_same54.o
 .group         0x0000000000000000        0xc ESF/mcu/src/startup_same54.o
 .group         0x0000000000000000        0xc ESF/mcu/src/startup_same54.o
 .group         0x0000000000000000        0xc ESF/mcu/src/startup_same54.o
 .group         0x0000000000000000        0xc ESF/mcu/src/startup_same54.o
 .group         0x0000000000000000        0xc ESF/mcu/src/startup_same54.o
 .group         0x0000000000000000        0xc ESF/mcu/src/startup_same54.o
 .group         0x0000000000000000        0xc ESF/mcu/src/startup_same54.o
 .group         0x0000000000000000        0xc ESF/mcu/src/startup_same54.o
 .group         0x0000000000000000        0xc ESF/mcu/src/startup_same54.o
 .group         0x0000000000000000        0xc ESF/mcu/src/startup_same54.o
 .group         0x0000000000000000        0xc ESF/mcu/src/startup_same54.o
 .group         0x0000000000000000        0xc ESF/mcu/src/startup_same54.o
 .group         0x0000000000000000        0xc ESF/mcu/src/startup_same54.o
 .group         0x0000000000000000        0xc ESF/mcu/src/startup_same54.o
 .group         0x0000000000000000        0xc ESF/mcu/src/startup_same54.o
 .group         0x0000000000000000        0xc ESF/mcu/src/startup_same54.o
 .group         0x0000000000000000        0xc ESF/mcu/src/startup_same54.o
 .group         0x0000000000000000        0xc ESF/mcu/src/startup_same54.o
 .group         0x0000000000000000        0xc ESF/mcu/src/startup_same54.o
 .group         0x0000000000000000        0xc ESF/mcu/src/startup_same54.o
 .group         0x0000000000000000        0xc ESF/mcu/src/startup_same54.o
 .group         0x0000000000000000        0xc ESF/mcu/src/startup_same54.o
 .group         0x0000000000000000        0xc ESF/mcu/src/startup_same54.o
 .group         0x0000000000000000        0xc ESF/mcu/src/startup_same54.o
 .group         0x0000000000000000        0xc ESF/mcu/src/startup_same54.o
 .group         0x0000000000000000        0xc ESF/mcu/src/startup_same54.o
 .group         0x0000000000000000        0xc ESF/mcu/src/startup_same54.o
 .group         0x0000000000000000        0xc ESF/mcu/src/startup_same54.o
 .group         0x0000000000000000        0xc ESF/mcu/src/startup_same54.o
 .group         0x0000000000000000        0xc ESF/mcu/src/startup_same54.o
 .group         0x0000000000000000        0xc ESF/mcu/src/startup_same54.o
 .group         0x0000000000000000        0xc ESF/mcu/src/startup_same54.o
 .group         0x0000000000000000        0xc ESF/mcu/src/startup_same54.o
 .group         0x0000000000000000        0xc ESF/mcu/src/startup_same54.o
 .group         0x0000000000000000        0xc ESF/mcu/src/startup_same54.o
 .group         0x0000000000000000        0xc ESF/mcu/src/startup_same54.o
 .group         0x0000000000000000        0xc ESF/mcu/src/startup_same54.o
 .group         0x0000000000000000        0xc ESF/mcu/src/startup_same54.o
 .group         0x0000000000000000        0xc ESF/mcu/src/startup_same54.o
 .group         0x0000000000000000        0xc ESF/mcu/src/startup_same54.o
 .group         0x0000000000000000        0xc ESF/mcu/src/startup_same54.o
 .group         0x0000000000000000        0xc ESF/mcu/src/startup_same54.o
 .group         0x0000000000000000        0xc ESF/mcu/src/startup_same54.o
 .group         0x0000000000000000        0xc ESF/mcu/src/startup_same54.o
 .group         0x0000000000000000        0xc ESF/mcu/src/startup_same54.o
 .group         0x0000000000000000        0xc ESF/mcu/src/startup_same54.o
 .group         0x0000000000000000        0xc ESF/mcu/src/startup_same54.o
 .group         0x0000000000000000        0xc ESF/mcu/src/startup_same54.o
 .group         0x0000000000000000        0xc ESF/mcu/src/startup_same54.o
 .group         0x0000000000000000        0xc ESF/mcu/src/startup_same54.o
 .group         0x0000000000000000        0xc ESF/mcu/src/startup_same54.o
 .group         0x0000000000000000        0xc ESF/mcu/src/startup_same54.o
 .group         0x0000000000000000        0xc ESF/mcu/src/startup_same54.o
 .group         0x0000000000000000        0xc ESF/mcu/src/startup_same54.o
 .group         0x0000000000000000        0xc ESF/mcu/src/startup_same54.o
 .group         0x0000000000000000        0xc ESF/mcu/src/startup_same54.o
 .group         0x0000000000000000        0xc ESF/mcu/src/startup_same54.o
 .group         0x0000000000000000        0xc ESF/mcu/src/startup_same54.o
 .group         0x0000000000000000        0xc ESF/mcu/src/startup_same54.o
 .group         0x0000000000000000        0xc ESF/mcu/src/startup_same54.o
 .group         0x0000000000000000        0xc ESF/mcu/src/startup_same54.o
 .group         0x0000000000000000        0xc ESF/mcu/src/startup_same54.o
 .group         0x0000000000000000        0xc ESF/mcu/src/startup_same54.o
 .group         0x0000000000000000        0xc ESF/mcu/src/startup_same54.o
 .group         0x0000000000000000        0xc ESF/mcu/src/startup_same54.o
 .group         0x0000000000000000        0xc ESF/mcu/src/startup_same54.o
 .group         0x0000000000000000        0xc ESF/mcu/src/startup_same54.o
 .group         0x0000000000000000        0xc ESF/mcu/src/startup_same54.o
 .group         0x0000000000000000        0xc ESF/mcu/src/startup_same54.o
 .group         0x0000000000000000        0xc ESF/mcu/src/startup_same54.o
 .group         0x0000000000000000        0xc ESF/mcu/src/startup_same54.o
 .group         0x0000000000000000        0xc ESF/mcu/src/startup_same54.o
 .group         0x0000000000000000        0xc ESF/mcu/src/startup_same54.o
 .group         0x0000000000000000        0xc ESF/mcu/src/startup_same54.o
 .group         0x0000000000000000        0xc ESF/mcu/src/startup_same54.o
 .group         0x0000000000000000        0xc ESF/mcu/src/startup_same54.o
 .group         0x0000000000000000        0xc ESF/mcu/src/startup_same54.o
 .group         0x0000000000000000        0xc ESF/mcu/src/startup_same54.o
 .group         0x0000000000000000        0xc ESF/mcu/src/startup_same54.o
 .group         0x0000000000000000        0xc ESF/mcu/src/startup_same54.o
 .group         0x0000000000000000        0xc ESF/mcu/src/startup_same54.o
 .group         0x0000000000000000        0xc ESF/mcu/src/startup_same54.o
 .group         0x0000000000000000        0xc ESF/mcu/src/startup_same54.o
 .text          0x0000000000000000        0x0 ESF/mcu/src/startup_same54.o
 .data          0x0000000000000000        0x0 ESF/mcu/src/startup_same54.o
 .bss           0x0000000000000000        0x0 ESF/mcu/src/startup_same54.o
 .group         0x0000000000000000        0xc ESF/mcu/src/system_same54.o
 .group         0x0000000000000000        0xc ESF/mcu/src/system_same54.o
 .group         0x0000000000000000        0xc ESF/mcu/src/system_same54.o
 .group         0x0000000000000000        0xc ESF/mcu/src/system_same54.o
 .group         0x0000000000000000        0xc ESF/mcu/src/system_same54.o
 .group         0x0000000000000000        0xc ESF/mcu/src/system_same54.o
 .group         0x0000000000000000        0xc ESF/mcu/src/system_same54.o
 .group         0x0000000000000000        0xc ESF/mcu/src/system_same54.o
 .group         0x0000000000000000        0xc ESF/mcu/src/system_same54.o
 .group         0x0000000000000000        0xc ESF/mcu/src/system_same54.o
 .group         0x0000000000000000        0xc ESF/mcu/src/system_same54.o
 .group         0x0000000000000000        0xc ESF/mcu/src/system_same54.o
 .group         0x0000000000000000        0xc ESF/mcu/src/system_same54.o
 .group         0x0000000000000000        0xc ESF/mcu/src/system_same54.o
 .group         0x0000000000000000        0xc ESF/mcu/src/system_same54.o
 .group         0x0000000000000000        0xc ESF/mcu/src/system_same54.o
 .group         0x0000000000000000        0xc ESF/mcu/src/system_same54.o
 .group         0x0000000000000000        0xc ESF/mcu/src/system_same54.o
 .group         0x0000000000000000        0xc ESF/mcu/src/system_same54.o
 .group         0x0000000000000000        0xc ESF/mcu/src/system_same54.o
 .group         0x0000000000000000        0xc ESF/mcu/src/system_same54.o
 .group         0x0000000000000000        0xc ESF/mcu/src/system_same54.o
 .group         0x0000000000000000        0xc ESF/mcu/src/system_same54.o
 .group         0x0000000000000000        0xc ESF/mcu/src/system_same54.o
 .group         0x0000000000000000        0xc ESF/mcu/src/system_same54.o
 .group         0x0000000000000000        0xc ESF/mcu/src/system_same54.o
 .group         0x0000000000000000        0xc ESF/mcu/src/system_same54.o
 .group         0x0000000000000000        0xc ESF/mcu/src/system_same54.o
 .group         0x0000000000000000        0xc ESF/mcu/src/system_same54.o
 .group         0x0000000000000000        0xc ESF/mcu/src/system_same54.o
 .group         0x0000000000000000        0xc ESF/mcu/src/system_same54.o
 .group         0x0000000000000000        0xc ESF/mcu/src/system_same54.o
 .group         0x0000000000000000        0xc ESF/mcu/src/system_same54.o
 .group         0x0000000000000000        0xc ESF/mcu/src/system_same54.o
 .group         0x0000000000000000        0xc ESF/mcu/src/system_same54.o
 .group         0x0000000000000000        0xc ESF/mcu/src/system_same54.o
 .group         0x0000000000000000        0xc ESF/mcu/src/system_same54.o
 .group         0x0000000000000000        0xc ESF/mcu/src/system_same54.o
 .group         0x0000000000000000        0xc ESF/mcu/src/system_same54.o
 .group         0x0000000000000000        0xc ESF/mcu/src/system_same54.o
 .group         0x0000000000000000        0xc ESF/mcu/src/system_same54.o
 .group         0x0000000000000000        0xc ESF/mcu/src/system_same54.o
 .group         0x0000000000000000        0xc ESF/mcu/src/system_same54.o
 .group         0x0000000000000000        0xc ESF/mcu/src/system_same54.o
 .group         0x0000000000000000        0xc ESF/mcu/src/system_same54.o
 .group         0x0000000000000000        0xc ESF/mcu/src/system_same54.o
 .group         0x0000000000000000        0xc ESF/mcu/src/system_same54.o
 .group         0x0000000000000000        0xc ESF/mcu/src/system_same54.o
 .group         0x0000000000000000        0xc ESF/mcu/src/system_same54.o
 .group         0x0000000000000000        0xc ESF/mcu/src/system_same54.o
 .group         0x0000000000000000        0xc ESF/mcu/src/system_same54.o
 .group         0x0000000000000000        0xc ESF/mcu/src/system_same54.o
 .group         0x0000000000000000        0xc ESF/mcu/src/system_same54.o
 .group         0x0000000000000000        0xc ESF/mcu/src/system_same54.o
 .group         0x0000000000000000        0xc ESF/mcu/src/system_same54.o
 .group         0x0000000000000000        0xc ESF/mcu/src/system_same54.o
 .group         0x0000000000000000        0xc ESF/mcu/src/system_same54.o
 .group         0x0000000000000000        0xc ESF/mcu/src/system_same54.o
 .group         0x0000000000000000        0xc ESF/mcu/src/system_same54.o
 .group         0x0000000000000000        0xc ESF/mcu/src/system_same54.o
 .group         0x0000000000000000        0xc ESF/mcu/src/system_same54.o
 .group         0x0000000000000000        0xc ESF/mcu/src/system_same54.o
 .group         0x0000000000000000        0xc ESF/mcu/src/system_same54.o
 .group         0x0000000000000000        0xc ESF/mcu/src/system_same54.o
 .group         0x0000000000000000        0xc ESF/mcu/src/system_same54.o
 .group         0x0000000000000000        0xc ESF/mcu/src/system_same54.o
 .group         0x0000000000000000        0xc ESF/mcu/src/system_same54.o
 .group         0x0000000000000000        0xc ESF/mcu/src/system_same54.o
 .group         0x0000000000000000        0xc ESF/mcu/src/system_same54.o
 .group         0x0000000000000000        0xc ESF/mcu/src/system_same54.o
 .group         0x0000000000000000        0xc ESF/mcu/src/system_same54.o
 .group         0x0000000000000000        0xc ESF/mcu/src/system_same54.o
 .group         0x0000000000000000        0xc ESF/mcu/src/system_same54.o
 .group         0x0000000000000000        0xc ESF/mcu/src/system_same54.o
 .group         0x0000000000000000        0xc ESF/mcu/src/system_same54.o
 .group         0x0000000000000000        0xc ESF/mcu/src/system_same54.o
 .group         0x0000000000000000        0xc ESF/mcu/src/system_same54.o
 .group         0x0000000000000000        0xc ESF/mcu/src/system_same54.o
 .group         0x0000000000000000        0xc ESF/mcu/src/system_same54.o
 .group         0x0000000000000000        0xc ESF/mcu/src/system_same54.o
 .group         0x0000000000000000        0xc ESF/mcu/src/system_same54.o
 .group         0x0000000000000000        0xc ESF/mcu/src/system_same54.o
 .group         0x0000000000000000        0xc ESF/mcu/src/system_same54.o
 .group         0x0000000000000000        0xc ESF/mcu/src/system_same54.o
 .group         0x0000000000000000        0xc ESF/mcu/src/system_same54.o
 .group         0x0000000000000000        0xc ESF/mcu/src/system_same54.o
 .group         0x0000000000000000        0xc ESF/mcu/src/system_same54.o
 .group         0x0000000000000000        0xc ESF/mcu/src/system_same54.o
 .group         0x0000000000000000        0xc ESF/mcu/src/system_same54.o
 .group         0x0000000000000000        0xc ESF/mcu/src/system_same54.o
 .group         0x0000000000000000        0xc ESF/mcu/src/system_same54.o
 .group         0x0000000000000000        0xc ESF/mcu/src/system_same54.o
 .group         0x0000000000000000        0xc ESF/mcu/src/system_same54.o
 .group         0x0000000000000000        0xc ESF/mcu/src/system_same54.o
 .group         0x0000000000000000        0xc ESF/mcu/src/system_same54.o
 .group         0x0000000000000000        0xc ESF/mcu/src/system_same54.o
 .group         0x0000000000000000        0xc ESF/mcu/src/system_same54.o
 .group         0x0000000000000000        0xc ESF/mcu/src/system_same54.o
 .group         0x0000000000000000        0xc ESF/mcu/src/system_same54.o
 .group         0x0000000000000000        0xc ESF/mcu/src/system_same54.o
 .group         0x0000000000000000        0xc ESF/mcu/src/system_same54.o
 .group         0x0000000000000000        0xc ESF/mcu/src/system_same54.o
 .group         0x0000000000000000        0xc ESF/mcu/src/system_same54.o
 .group         0x0000000000000000        0xc ESF/mcu/src/system_same54.o
 .group         0x0000000000000000        0xc ESF/mcu/src/system_same54.o
 .group         0x0000000000000000        0xc ESF/mcu/src/system_same54.o
 .group         0x0000000000000000        0xc ESF/mcu/src/system_same54.o
 .group         0x0000000000000000        0xc ESF/mcu/src/system_same54.o
 .group         0x0000000000000000        0xc ESF/mcu/src/system_same54.o
 .group         0x0000000000000000        0xc ESF/mcu/src/system_same54.o
 .group         0x0000000000000000        0xc ESF/mcu/src/system_same54.o
 .group         0x0000000000000000        0xc ESF/mcu/src/system_same54.o
 .group         0x0000000000000000        0xc ESF/mcu/src/system_same54.o
 .group         0x0000000000000000        0xc ESF/mcu/src/system_same54.o
 .text          0x0000000000000000        0x0 ESF/mcu/src/system_same54.o
 .data          0x0000000000000000        0x4 ESF/mcu/src/system_same54.o
 .bss           0x0000000000000000        0x0 ESF/mcu/src/system_same54.o
 .text.SystemInit
                0x0000000000000000       0x10 ESF/mcu/src/system_same54.o
 .text.SystemCoreClockUpdate
                0x0000000000000000       0x10 ESF/mcu/src/system_same54.o
 .debug_info    0x0000000000000000       0xc2 ESF/mcu/src/system_same54.o
 .debug_abbrev  0x0000000000000000       0x92 ESF/mcu/src/system_same54.o
 .debug_aranges
                0x0000000000000000       0x20 ESF/mcu/src/system_same54.o
 .debug_ranges  0x0000000000000000       0x10 ESF/mcu/src/system_same54.o
 .debug_macro   0x0000000000000000      0x4b8 ESF/mcu/src/system_same54.o
 .debug_macro   0x0000000000000000      0xa78 ESF/mcu/src/system_same54.o
 .debug_macro   0x0000000000000000       0x22 ESF/mcu/src/system_same54.o
 .debug_macro   0x0000000000000000       0x8e ESF/mcu/src/system_same54.o
 .debug_macro   0x0000000000000000       0x51 ESF/mcu/src/system_same54.o
 .debug_macro   0x0000000000000000      0x103 ESF/mcu/src/system_same54.o
 .debug_macro   0x0000000000000000       0x6a ESF/mcu/src/system_same54.o
 .debug_macro   0x0000000000000000      0x1df ESF/mcu/src/system_same54.o
 .debug_macro   0x0000000000000000       0x4e ESF/mcu/src/system_same54.o
 .debug_macro   0x0000000000000000       0x1c ESF/mcu/src/system_same54.o
 .debug_macro   0x0000000000000000       0x22 ESF/mcu/src/system_same54.o
 .debug_macro   0x0000000000000000       0xd9 ESF/mcu/src/system_same54.o
 .debug_macro   0x0000000000000000     0x102d ESF/mcu/src/system_same54.o
 .debug_macro   0x0000000000000000      0x11f ESF/mcu/src/system_same54.o
 .debug_macro   0x0000000000000000      0x706 ESF/mcu/src/system_same54.o
 .debug_macro   0x0000000000000000      0xb5b ESF/mcu/src/system_same54.o
 .debug_macro   0x0000000000000000      0x3c0 ESF/mcu/src/system_same54.o
 .debug_macro   0x0000000000000000     0x2d61 ESF/mcu/src/system_same54.o
 .debug_macro   0x0000000000000000      0x336 ESF/mcu/src/system_same54.o
 .debug_macro   0x0000000000000000      0x3b7 ESF/mcu/src/system_same54.o
 .debug_macro   0x0000000000000000      0x668 ESF/mcu/src/system_same54.o
 .debug_macro   0x0000000000000000     0x143f ESF/mcu/src/system_same54.o
 .debug_macro   0x0000000000000000      0x651 ESF/mcu/src/system_same54.o
 .debug_macro   0x0000000000000000      0x67b ESF/mcu/src/system_same54.o
 .debug_macro   0x0000000000000000      0x6d7 ESF/mcu/src/system_same54.o
 .debug_macro   0x0000000000000000      0x172 ESF/mcu/src/system_same54.o
 .debug_macro   0x0000000000000000      0x395 ESF/mcu/src/system_same54.o
 .debug_macro   0x0000000000000000     0x19dd ESF/mcu/src/system_same54.o
 .debug_macro   0x0000000000000000       0x3a ESF/mcu/src/system_same54.o
 .debug_macro   0x0000000000000000      0x72a ESF/mcu/src/system_same54.o
 .debug_macro   0x0000000000000000      0xb12 ESF/mcu/src/system_same54.o
 .debug_macro   0x0000000000000000      0x5d7 ESF/mcu/src/system_same54.o
 .debug_macro   0x0000000000000000      0xbc0 ESF/mcu/src/system_same54.o
 .debug_macro   0x0000000000000000      0x9b9 ESF/mcu/src/system_same54.o
 .debug_macro   0x0000000000000000      0x2a3 ESF/mcu/src/system_same54.o
 .debug_macro   0x0000000000000000      0x8cb ESF/mcu/src/system_same54.o
 .debug_macro   0x0000000000000000      0x1ea ESF/mcu/src/system_same54.o
 .debug_macro   0x0000000000000000      0x8f4 ESF/mcu/src/system_same54.o
 .debug_macro   0x0000000000000000      0x216 ESF/mcu/src/system_same54.o
 .debug_macro   0x0000000000000000      0x3f9 ESF/mcu/src/system_same54.o
 .debug_macro   0x0000000000000000      0x620 ESF/mcu/src/system_same54.o
 .debug_macro   0x0000000000000000      0x10d ESF/mcu/src/system_same54.o
 .debug_macro   0x0000000000000000       0xb8 ESF/mcu/src/system_same54.o
 .debug_macro   0x0000000000000000     0x1df7 ESF/mcu/src/system_same54.o
 .debug_macro   0x0000000000000000     0x2e69 ESF/mcu/src/system_same54.o
 .debug_macro   0x0000000000000000     0x11ed ESF/mcu/src/system_same54.o
 .debug_macro   0x0000000000000000      0x50e ESF/mcu/src/system_same54.o
 .debug_macro   0x0000000000000000      0x930 ESF/mcu/src/system_same54.o
 .debug_macro   0x0000000000000000     0x1ad8 ESF/mcu/src/system_same54.o
 .debug_macro   0x0000000000000000       0xe7 ESF/mcu/src/system_same54.o
 .debug_macro   0x0000000000000000     0x13e6 ESF/mcu/src/system_same54.o
 .debug_macro   0x0000000000000000      0x36a ESF/mcu/src/system_same54.o
 .debug_macro   0x0000000000000000       0x94 ESF/mcu/src/system_same54.o
 .debug_macro   0x0000000000000000       0xdc ESF/mcu/src/system_same54.o
 .debug_macro   0x0000000000000000       0xe2 ESF/mcu/src/system_same54.o
 .debug_macro   0x0000000000000000       0xdc ESF/mcu/src/system_same54.o
 .debug_macro   0x0000000000000000      0x149 ESF/mcu/src/system_same54.o
 .debug_macro   0x0000000000000000      0x149 ESF/mcu/src/system_same54.o
 .debug_macro   0x0000000000000000       0x46 ESF/mcu/src/system_same54.o
 .debug_macro   0x0000000000000000       0x4c ESF/mcu/src/system_same54.o
 .debug_macro   0x0000000000000000       0xc4 ESF/mcu/src/system_same54.o
 .debug_macro   0x0000000000000000      0x7d5 ESF/mcu/src/system_same54.o
 .debug_macro   0x0000000000000000       0xb8 ESF/mcu/src/system_same54.o
 .debug_macro   0x0000000000000000       0x7c ESF/mcu/src/system_same54.o
 .debug_macro   0x0000000000000000      0xc20 ESF/mcu/src/system_same54.o
 .debug_macro   0x0000000000000000       0x46 ESF/mcu/src/system_same54.o
 .debug_macro   0x0000000000000000      0x25b ESF/mcu/src/system_same54.o
 .debug_macro   0x0000000000000000      0x31a ESF/mcu/src/system_same54.o
 .debug_macro   0x0000000000000000      0x170 ESF/mcu/src/system_same54.o
 .debug_macro   0x0000000000000000       0x7c ESF/mcu/src/system_same54.o
 .debug_macro   0x0000000000000000       0xbe ESF/mcu/src/system_same54.o
 .debug_macro   0x0000000000000000       0x4c ESF/mcu/src/system_same54.o
 .debug_macro   0x0000000000000000       0x82 ESF/mcu/src/system_same54.o
 .debug_macro   0x0000000000000000      0x1a3 ESF/mcu/src/system_same54.o
 .debug_macro   0x0000000000000000       0x46 ESF/mcu/src/system_same54.o
 .debug_macro   0x0000000000000000       0x6a ESF/mcu/src/system_same54.o
 .debug_macro   0x0000000000000000       0x46 ESF/mcu/src/system_same54.o
 .debug_macro   0x0000000000000000       0x88 ESF/mcu/src/system_same54.o
 .debug_macro   0x0000000000000000       0x46 ESF/mcu/src/system_same54.o
 .debug_macro   0x0000000000000000      0x24e ESF/mcu/src/system_same54.o
 .debug_macro   0x0000000000000000       0x1c ESF/mcu/src/system_same54.o
 .debug_macro   0x0000000000000000       0x76 ESF/mcu/src/system_same54.o
 .debug_macro   0x0000000000000000       0x3a ESF/mcu/src/system_same54.o
 .debug_macro   0x0000000000000000       0x2e ESF/mcu/src/system_same54.o
 .debug_macro   0x0000000000000000      0x196 ESF/mcu/src/system_same54.o
 .debug_macro   0x0000000000000000      0x16f ESF/mcu/src/system_same54.o
 .debug_macro   0x0000000000000000      0x16f ESF/mcu/src/system_same54.o
 .debug_macro   0x0000000000000000      0x25d ESF/mcu/src/system_same54.o
 .debug_macro   0x0000000000000000      0x25d ESF/mcu/src/system_same54.o
 .debug_macro   0x0000000000000000      0x25d ESF/mcu/src/system_same54.o
 .debug_macro   0x0000000000000000      0x25d ESF/mcu/src/system_same54.o
 .debug_macro   0x0000000000000000      0x25d ESF/mcu/src/system_same54.o
 .debug_macro   0x0000000000000000      0x25d ESF/mcu/src/system_same54.o
 .debug_macro   0x0000000000000000      0x25d ESF/mcu/src/system_same54.o
 .debug_macro   0x0000000000000000      0x25d ESF/mcu/src/system_same54.o
 .debug_macro   0x0000000000000000       0x52 ESF/mcu/src/system_same54.o
 .debug_macro   0x0000000000000000       0xfa ESF/mcu/src/system_same54.o
 .debug_macro   0x0000000000000000       0xfa ESF/mcu/src/system_same54.o
 .debug_macro   0x0000000000000000       0xfa ESF/mcu/src/system_same54.o
 .debug_macro   0x0000000000000000       0xfa ESF/mcu/src/system_same54.o
 .debug_macro   0x0000000000000000       0xfa ESF/mcu/src/system_same54.o
 .debug_macro   0x0000000000000000       0xfa ESF/mcu/src/system_same54.o
 .debug_macro   0x0000000000000000       0xfa ESF/mcu/src/system_same54.o
 .debug_macro   0x0000000000000000       0xfa ESF/mcu/src/system_same54.o
 .debug_macro   0x0000000000000000      0x148 ESF/mcu/src/system_same54.o
 .debug_macro   0x0000000000000000      0x124 ESF/mcu/src/system_same54.o
 .debug_macro   0x0000000000000000      0x106 ESF/mcu/src/system_same54.o
 .debug_macro   0x0000000000000000       0xee ESF/mcu/src/system_same54.o
 .debug_macro   0x0000000000000000       0xee ESF/mcu/src/system_same54.o
 .debug_macro   0x0000000000000000       0x2e ESF/mcu/src/system_same54.o
 .debug_macro   0x0000000000000000      0x46a ESF/mcu/src/system_same54.o
 .debug_macro   0x0000000000000000       0x3a ESF/mcu/src/system_same54.o
 .debug_macro   0x0000000000000000      0x59f ESF/mcu/src/system_same54.o
 .debug_macro   0x0000000000000000     0x4ff3 ESF/mcu/src/system_same54.o
 .debug_macro   0x0000000000000000       0xcf ESF/mcu/src/system_same54.o
 .debug_line    0x0000000000000000      0x62c ESF/mcu/src/system_same54.o
 .debug_str     0x0000000000000000    0xf088b ESF/mcu/src/system_same54.o
 .comment       0x0000000000000000       0x1f ESF/mcu/src/system_same54.o
 .debug_frame   0x0000000000000000       0x30 ESF/mcu/src/system_same54.o
 .ARM.attributes
                0x0000000000000000       0x32 ESF/mcu/src/system_same54.o
 .group         0x0000000000000000        0xc src/main.o
 .group         0x0000000000000000        0xc src/main.o
 .group         0x0000000000000000        0xc src/main.o
 .group         0x0000000000000000        0xc src/main.o
 .group         0x0000000000000000        0xc src/main.o
 .group         0x0000000000000000        0xc src/main.o
 .group         0x0000000000000000        0xc src/main.o
 .group         0x0000000000000000        0xc src/main.o
 .group         0x0000000000000000        0xc src/main.o
 .group         0x0000000000000000        0xc src/main.o
 .group         0x0000000000000000        0xc src/main.o
 .group         0x0000000000000000        0xc src/main.o
 .group         0x0000000000000000        0xc src/main.o
 .group         0x0000000000000000        0xc src/main.o
 .group         0x0000000000000000        0xc src/main.o
 .group         0x0000000000000000        0xc src/main.o
 .group         0x0000000000000000        0xc src/main.o
 .group         0x0000000000000000        0xc src/main.o
 .group         0x0000000000000000        0xc src/main.o
 .group         0x0000000000000000        0xc src/main.o
 .group         0x0000000000000000        0xc src/main.o
 .group         0x0000000000000000        0xc src/main.o
 .group         0x0000000000000000        0xc src/main.o
 .group         0x0000000000000000        0xc src/main.o
 .group         0x0000000000000000        0xc src/main.o
 .group         0x0000000000000000        0xc src/main.o
 .group         0x0000000000000000        0xc src/main.o
 .group         0x0000000000000000        0xc src/main.o
 .group         0x0000000000000000        0xc src/main.o
 .group         0x0000000000000000        0xc src/main.o
 .group         0x0000000000000000        0xc src/main.o
 .group         0x0000000000000000        0xc src/main.o
 .group         0x0000000000000000        0xc src/main.o
 .group         0x0000000000000000        0xc src/main.o
 .group         0x0000000000000000        0xc src/main.o
 .group         0x0000000000000000        0xc src/main.o
 .group         0x0000000000000000        0xc src/main.o
 .group         0x0000000000000000        0xc src/main.o
 .group         0x0000000000000000        0xc src/main.o
 .group         0x0000000000000000        0xc src/main.o
 .group         0x0000000000000000        0xc src/main.o
 .group         0x0000000000000000        0xc src/main.o
 .group         0x0000000000000000        0xc src/main.o
 .group         0x0000000000000000        0xc src/main.o
 .group         0x0000000000000000        0xc src/main.o
 .group         0x0000000000000000        0xc src/main.o
 .group         0x0000000000000000        0xc src/main.o
 .group         0x0000000000000000        0xc src/main.o
 .group         0x0000000000000000        0xc src/main.o
 .group         0x0000000000000000        0xc src/main.o
 .group         0x0000000000000000        0xc src/main.o
 .group         0x0000000000000000        0xc src/main.o
 .group         0x0000000000000000        0xc src/main.o
 .group         0x0000000000000000        0xc src/main.o
 .group         0x0000000000000000        0xc src/main.o
 .group         0x0000000000000000        0xc src/main.o
 .group         0x0000000000000000        0xc src/main.o
 .group         0x0000000000000000        0xc src/main.o
 .group         0x0000000000000000        0xc src/main.o
 .group         0x0000000000000000        0xc src/main.o
 .group         0x0000000000000000        0xc src/main.o
 .group         0x0000000000000000        0xc src/main.o
 .group         0x0000000000000000        0xc src/main.o
 .group         0x0000000000000000        0xc src/main.o
 .group         0x0000000000000000        0xc src/main.o
 .group         0x0000000000000000        0xc src/main.o
 .group         0x0000000000000000        0xc src/main.o
 .group         0x0000000000000000        0xc src/main.o
 .group         0x0000000000000000        0xc src/main.o
 .group         0x0000000000000000        0xc src/main.o
 .group         0x0000000000000000        0xc src/main.o
 .group         0x0000000000000000        0xc src/main.o
 .group         0x0000000000000000        0xc src/main.o
 .group         0x0000000000000000        0xc src/main.o
 .group         0x0000000000000000        0xc src/main.o
 .group         0x0000000000000000        0xc src/main.o
 .group         0x0000000000000000        0xc src/main.o
 .group         0x0000000000000000        0xc src/main.o
 .group         0x0000000000000000        0xc src/main.o
 .group         0x0000000000000000        0xc src/main.o
 .group         0x0000000000000000        0xc src/main.o
 .group         0x0000000000000000        0xc src/main.o
 .group         0x0000000000000000        0xc src/main.o
 .group         0x0000000000000000        0xc src/main.o
 .group         0x0000000000000000        0xc src/main.o
 .group         0x0000000000000000        0xc src/main.o
 .group         0x0000000000000000        0xc src/main.o
 .group         0x0000000000000000        0xc src/main.o
 .group         0x0000000000000000        0xc src/main.o
 .group         0x0000000000000000        0xc src/main.o
 .group         0x0000000000000000        0xc src/main.o
 .group         0x0000000000000000        0xc src/main.o
 .group         0x0000000000000000        0xc src/main.o
 .group         0x0000000000000000        0xc src/main.o
 .group         0x0000000000000000        0xc src/main.o
 .group         0x0000000000000000        0xc src/main.o
 .group         0x0000000000000000        0xc src/main.o
 .group         0x0000000000000000        0xc src/main.o
 .group         0x0000000000000000        0xc src/main.o
 .group         0x0000000000000000        0xc src/main.o
 .group         0x0000000000000000        0xc src/main.o
 .group         0x0000000000000000        0xc src/main.o
 .group         0x0000000000000000        0xc src/main.o
 .group         0x0000000000000000        0xc src/main.o
 .group         0x0000000000000000        0xc src/main.o
 .group         0x0000000000000000        0xc src/main.o
 .group         0x0000000000000000        0xc src/main.o
 .group         0x0000000000000000        0xc src/main.o
 .group         0x0000000000000000        0xc src/main.o
 .group         0x0000000000000000        0xc src/main.o
 .group         0x0000000000000000        0xc src/main.o
 .group         0x0000000000000000        0xc src/main.o
 .group         0x0000000000000000        0xc src/main.o
 .group         0x0000000000000000        0xc src/main.o
 .text          0x0000000000000000        0x0 src/main.o
 .data          0x0000000000000000        0x0 src/main.o
 .bss           0x0000000000000000        0x0 src/main.o
 .debug_macro   0x0000000000000000      0xa78 src/main.o
 .debug_macro   0x0000000000000000       0x22 src/main.o
 .debug_macro   0x0000000000000000       0x8e src/main.o
 .debug_macro   0x0000000000000000       0x51 src/main.o
 .debug_macro   0x0000000000000000      0x103 src/main.o
 .debug_macro   0x0000000000000000       0x6a src/main.o
 .debug_macro   0x0000000000000000      0x1df src/main.o
 .debug_macro   0x0000000000000000       0x4e src/main.o
 .debug_macro   0x0000000000000000       0x1c src/main.o
 .debug_macro   0x0000000000000000       0x22 src/main.o
 .debug_macro   0x0000000000000000       0xd9 src/main.o
 .debug_macro   0x0000000000000000     0x102d src/main.o
 .debug_macro   0x0000000000000000      0x11f src/main.o
 .debug_macro   0x0000000000000000      0x706 src/main.o
 .debug_macro   0x0000000000000000      0xb5b src/main.o
 .debug_macro   0x0000000000000000      0x3c0 src/main.o
 .debug_macro   0x0000000000000000     0x2d61 src/main.o
 .debug_macro   0x0000000000000000      0x336 src/main.o
 .debug_macro   0x0000000000000000      0x3b7 src/main.o
 .debug_macro   0x0000000000000000      0x668 src/main.o
 .debug_macro   0x0000000000000000     0x143f src/main.o
 .debug_macro   0x0000000000000000      0x651 src/main.o
 .debug_macro   0x0000000000000000      0x67b src/main.o
 .debug_macro   0x0000000000000000      0x6d7 src/main.o
 .debug_macro   0x0000000000000000      0x172 src/main.o
 .debug_macro   0x0000000000000000      0x395 src/main.o
 .debug_macro   0x0000000000000000     0x19dd src/main.o
 .debug_macro   0x0000000000000000       0x3a src/main.o
 .debug_macro   0x0000000000000000      0x72a src/main.o
 .debug_macro   0x0000000000000000      0xb12 src/main.o
 .debug_macro   0x0000000000000000      0x5d7 src/main.o
 .debug_macro   0x0000000000000000      0xbc0 src/main.o
 .debug_macro   0x0000000000000000      0x9b9 src/main.o
 .debug_macro   0x0000000000000000      0x2a3 src/main.o
 .debug_macro   0x0000000000000000      0x8cb src/main.o
 .debug_macro   0x0000000000000000      0x1ea src/main.o
 .debug_macro   0x0000000000000000      0x8f4 src/main.o
 .debug_macro   0x0000000000000000      0x216 src/main.o
 .debug_macro   0x0000000000000000      0x3f9 src/main.o
 .debug_macro   0x0000000000000000      0x620 src/main.o
 .debug_macro   0x0000000000000000      0x10d src/main.o
 .debug_macro   0x0000000000000000       0xb8 src/main.o
 .debug_macro   0x0000000000000000     0x1df7 src/main.o
 .debug_macro   0x0000000000000000     0x2e69 src/main.o
 .debug_macro   0x0000000000000000     0x11ed src/main.o
 .debug_macro   0x0000000000000000      0x50e src/main.o
 .debug_macro   0x0000000000000000      0x930 src/main.o
 .debug_macro   0x0000000000000000     0x1ad8 src/main.o
 .debug_macro   0x0000000000000000       0xe7 src/main.o
 .debug_macro   0x0000000000000000     0x13e6 src/main.o
 .debug_macro   0x0000000000000000      0x36a src/main.o
 .debug_macro   0x0000000000000000       0x94 src/main.o
 .debug_macro   0x0000000000000000       0xdc src/main.o
 .debug_macro   0x0000000000000000       0xe2 src/main.o
 .debug_macro   0x0000000000000000       0xdc src/main.o
 .debug_macro   0x0000000000000000      0x149 src/main.o
 .debug_macro   0x0000000000000000      0x149 src/main.o
 .debug_macro   0x0000000000000000       0x46 src/main.o
 .debug_macro   0x0000000000000000       0x4c src/main.o
 .debug_macro   0x0000000000000000       0xc4 src/main.o
 .debug_macro   0x0000000000000000      0x7d5 src/main.o
 .debug_macro   0x0000000000000000       0xb8 src/main.o
 .debug_macro   0x0000000000000000       0x7c src/main.o
 .debug_macro   0x0000000000000000      0xc20 src/main.o
 .debug_macro   0x0000000000000000       0x46 src/main.o
 .debug_macro   0x0000000000000000      0x25b src/main.o
 .debug_macro   0x0000000000000000      0x31a src/main.o
 .debug_macro   0x0000000000000000      0x170 src/main.o
 .debug_macro   0x0000000000000000       0x7c src/main.o
 .debug_macro   0x0000000000000000       0xbe src/main.o
 .debug_macro   0x0000000000000000       0x4c src/main.o
 .debug_macro   0x0000000000000000       0x82 src/main.o
 .debug_macro   0x0000000000000000      0x1a3 src/main.o
 .debug_macro   0x0000000000000000       0x46 src/main.o
 .debug_macro   0x0000000000000000       0x6a src/main.o
 .debug_macro   0x0000000000000000       0x46 src/main.o
 .debug_macro   0x0000000000000000       0x88 src/main.o
 .debug_macro   0x0000000000000000       0x46 src/main.o
 .debug_macro   0x0000000000000000      0x24e src/main.o
 .debug_macro   0x0000000000000000       0x1c src/main.o
 .debug_macro   0x0000000000000000       0x76 src/main.o
 .debug_macro   0x0000000000000000       0x3a src/main.o
 .debug_macro   0x0000000000000000       0x2e src/main.o
 .debug_macro   0x0000000000000000      0x196 src/main.o
 .debug_macro   0x0000000000000000      0x16f src/main.o
 .debug_macro   0x0000000000000000      0x16f src/main.o
 .debug_macro   0x0000000000000000      0x25d src/main.o
 .debug_macro   0x0000000000000000      0x25d src/main.o
 .debug_macro   0x0000000000000000      0x25d src/main.o
 .debug_macro   0x0000000000000000      0x25d src/main.o
 .debug_macro   0x0000000000000000      0x25d src/main.o
 .debug_macro   0x0000000000000000      0x25d src/main.o
 .debug_macro   0x0000000000000000      0x25d src/main.o
 .debug_macro   0x0000000000000000      0x25d src/main.o
 .debug_macro   0x0000000000000000       0x52 src/main.o
 .debug_macro   0x0000000000000000       0xfa src/main.o
 .debug_macro   0x0000000000000000       0xfa src/main.o
 .debug_macro   0x0000000000000000       0xfa src/main.o
 .debug_macro   0x0000000000000000       0xfa src/main.o
 .debug_macro   0x0000000000000000       0xfa src/main.o
 .debug_macro   0x0000000000000000       0xfa src/main.o
 .debug_macro   0x0000000000000000       0xfa src/main.o
 .debug_macro   0x0000000000000000       0xfa src/main.o
 .debug_macro   0x0000000000000000      0x148 src/main.o
 .debug_macro   0x0000000000000000      0x124 src/main.o
 .debug_macro   0x0000000000000000      0x106 src/main.o
 .debug_macro   0x0000000000000000       0xee src/main.o
 .debug_macro   0x0000000000000000       0xee src/main.o
 .debug_macro   0x0000000000000000       0x2e src/main.o
 .debug_macro   0x0000000000000000      0x46a src/main.o
 .debug_macro   0x0000000000000000       0x3a src/main.o
 .debug_macro   0x0000000000000000      0x59f src/main.o
 .debug_macro   0x0000000000000000     0x4ff3 src/main.o
 .debug_macro   0x0000000000000000       0xcf src/main.o
 .text          0x0000000000000000        0x0 /usr/lib/gcc/arm-none-eabi/10.2.0/../../../../arm-none-eabi/lib/thumb/v7e-m/nofp/libc_nano.a(lib_a-atexit.o)
 .data          0x0000000000000000        0x0 /usr/lib/gcc/arm-none-eabi/10.2.0/../../../../arm-none-eabi/lib/thumb/v7e-m/nofp/libc_nano.a(lib_a-atexit.o)
 .bss           0x0000000000000000        0x0 /usr/lib/gcc/arm-none-eabi/10.2.0/../../../../arm-none-eabi/lib/thumb/v7e-m/nofp/libc_nano.a(lib_a-atexit.o)
 .text.atexit   0x0000000000000000        0xc /usr/lib/gcc/arm-none-eabi/10.2.0/../../../../arm-none-eabi/lib/thumb/v7e-m/nofp/libc_nano.a(lib_a-atexit.o)
 .debug_frame   0x0000000000000000       0x20 /usr/lib/gcc/arm-none-eabi/10.2.0/../../../../arm-none-eabi/lib/thumb/v7e-m/nofp/libc_nano.a(lib_a-atexit.o)
 .ARM.attributes
                0x0000000000000000       0x2e /usr/lib/gcc/arm-none-eabi/10.2.0/../../../../arm-none-eabi/lib/thumb/v7e-m/nofp/libc_nano.a(lib_a-atexit.o)
 .text          0x0000000000000000        0x0 /usr/lib/gcc/arm-none-eabi/10.2.0/../../../../arm-none-eabi/lib/thumb/v7e-m/nofp/libc_nano.a(lib_a-exit.o)
 .data          0x0000000000000000        0x0 /usr/lib/gcc/arm-none-eabi/10.2.0/../../../../arm-none-eabi/lib/thumb/v7e-m/nofp/libc_nano.a(lib_a-exit.o)
 .bss           0x0000000000000000        0x0 /usr/lib/gcc/arm-none-eabi/10.2.0/../../../../arm-none-eabi/lib/thumb/v7e-m/nofp/libc_nano.a(lib_a-exit.o)
 .text.exit     0x0000000000000000       0x28 /usr/lib/gcc/arm-none-eabi/10.2.0/../../../../arm-none-eabi/lib/thumb/v7e-m/nofp/libc_nano.a(lib_a-exit.o)
 .debug_frame   0x0000000000000000       0x28 /usr/lib/gcc/arm-none-eabi/10.2.0/../../../../arm-none-eabi/lib/thumb/v7e-m/nofp/libc_nano.a(lib_a-exit.o)
 .ARM.attributes
                0x0000000000000000       0x2e /usr/lib/gcc/arm-none-eabi/10.2.0/../../../../arm-none-eabi/lib/thumb/v7e-m/nofp/libc_nano.a(lib_a-exit.o)
 .text          0x0000000000000000        0x0 /usr/lib/gcc/arm-none-eabi/10.2.0/../../../../arm-none-eabi/lib/thumb/v7e-m/nofp/libc_nano.a(lib_a-fini.o)
 .data          0x0000000000000000        0x0 /usr/lib/gcc/arm-none-eabi/10.2.0/../../../../arm-none-eabi/lib/thumb/v7e-m/nofp/libc_nano.a(lib_a-fini.o)
 .bss           0x0000000000000000        0x0 /usr/lib/gcc/arm-none-eabi/10.2.0/../../../../arm-none-eabi/lib/thumb/v7e-m/nofp/libc_nano.a(lib_a-fini.o)
 .text.__libc_fini_array
                0x0000000000000000       0x28 /usr/lib/gcc/arm-none-eabi/10.2.0/../../../../arm-none-eabi/lib/thumb/v7e-m/nofp/libc_nano.a(lib_a-fini.o)
 .debug_frame   0x0000000000000000       0x38 /usr/lib/gcc/arm-none-eabi/10.2.0/../../../../arm-none-eabi/lib/thumb/v7e-m/nofp/libc_nano.a(lib_a-fini.o)
 .ARM.attributes
                0x0000000000000000       0x2e /usr/lib/gcc/arm-none-eabi/10.2.0/../../../../arm-none-eabi/lib/thumb/v7e-m/nofp/libc_nano.a(lib_a-fini.o)
 .text          0x0000000000000000        0x0 /usr/lib/gcc/arm-none-eabi/10.2.0/../../../../arm-none-eabi/lib/thumb/v7e-m/nofp/libc_nano.a(lib_a-impure.o)
 .data          0x0000000000000000        0x0 /usr/lib/gcc/arm-none-eabi/10.2.0/../../../../arm-none-eabi/lib/thumb/v7e-m/nofp/libc_nano.a(lib_a-impure.o)
 .bss           0x0000000000000000        0x0 /usr/lib/gcc/arm-none-eabi/10.2.0/../../../../arm-none-eabi/lib/thumb/v7e-m/nofp/libc_nano.a(lib_a-impure.o)
 .data._impure_ptr
                0x0000000000000000        0x4 /usr/lib/gcc/arm-none-eabi/10.2.0/../../../../arm-none-eabi/lib/thumb/v7e-m/nofp/libc_nano.a(lib_a-impure.o)
 .data.impure_data
                0x0000000000000000       0x60 /usr/lib/gcc/arm-none-eabi/10.2.0/../../../../arm-none-eabi/lib/thumb/v7e-m/nofp/libc_nano.a(lib_a-impure.o)
 .rodata._global_impure_ptr
                0x0000000000000000        0x4 /usr/lib/gcc/arm-none-eabi/10.2.0/../../../../arm-none-eabi/lib/thumb/v7e-m/nofp/libc_nano.a(lib_a-impure.o)
 .ARM.attributes
                0x0000000000000000       0x2e /usr/lib/gcc/arm-none-eabi/10.2.0/../../../../arm-none-eabi/lib/thumb/v7e-m/nofp/libc_nano.a(lib_a-impure.o)
 .text          0x0000000000000000        0x0 /usr/lib/gcc/arm-none-eabi/10.2.0/../../../../arm-none-eabi/lib/thumb/v7e-m/nofp/libc_nano.a(lib_a-init.o)
 .data          0x0000000000000000        0x0 /usr/lib/gcc/arm-none-eabi/10.2.0/../../../../arm-none-eabi/lib/thumb/v7e-m/nofp/libc_nano.a(lib_a-init.o)
 .bss           0x0000000000000000        0x0 /usr/lib/gcc/arm-none-eabi/10.2.0/../../../../arm-none-eabi/lib/thumb/v7e-m/nofp/libc_nano.a(lib_a-init.o)
 .text          0x0000000000000000        0x0 /usr/lib/gcc/arm-none-eabi/10.2.0/../../../../arm-none-eabi/lib/thumb/v7e-m/nofp/libc_nano.a(lib_a-memcpy-stub.o)
 .data          0x0000000000000000        0x0 /usr/lib/gcc/arm-none-eabi/10.2.0/../../../../arm-none-eabi/lib/thumb/v7e-m/nofp/libc_nano.a(lib_a-memcpy-stub.o)
 .bss           0x0000000000000000        0x0 /usr/lib/gcc/arm-none-eabi/10.2.0/../../../../arm-none-eabi/lib/thumb/v7e-m/nofp/libc_nano.a(lib_a-memcpy-stub.o)
 .text          0x0000000000000000        0x0 /usr/lib/gcc/arm-none-eabi/10.2.0/../../../../arm-none-eabi/lib/thumb/v7e-m/nofp/libc_nano.a(lib_a-memset.o)
 .data          0x0000000000000000        0x0 /usr/lib/gcc/arm-none-eabi/10.2.0/../../../../arm-none-eabi/lib/thumb/v7e-m/nofp/libc_nano.a(lib_a-memset.o)
 .bss           0x0000000000000000        0x0 /usr/lib/gcc/arm-none-eabi/10.2.0/../../../../arm-none-eabi/lib/thumb/v7e-m/nofp/libc_nano.a(lib_a-memset.o)
 .text          0x0000000000000000        0x0 /usr/lib/gcc/arm-none-eabi/10.2.0/../../../../arm-none-eabi/lib/thumb/v7e-m/nofp/libc_nano.a(lib_a-__atexit.o)
 .data          0x0000000000000000        0x0 /usr/lib/gcc/arm-none-eabi/10.2.0/../../../../arm-none-eabi/lib/thumb/v7e-m/nofp/libc_nano.a(lib_a-__atexit.o)
 .bss           0x0000000000000000        0x0 /usr/lib/gcc/arm-none-eabi/10.2.0/../../../../arm-none-eabi/lib/thumb/v7e-m/nofp/libc_nano.a(lib_a-__atexit.o)
 .text.__register_exitproc
                0x0000000000000000       0xc4 /usr/lib/gcc/arm-none-eabi/10.2.0/../../../../arm-none-eabi/lib/thumb/v7e-m/nofp/libc_nano.a(lib_a-__atexit.o)
 .bss._global_atexit0
                0x0000000000000000       0x8c /usr/lib/gcc/arm-none-eabi/10.2.0/../../../../arm-none-eabi/lib/thumb/v7e-m/nofp/libc_nano.a(lib_a-__atexit.o)
 .data.__atexit_dummy
                0x0000000000000000        0x4 /usr/lib/gcc/arm-none-eabi/10.2.0/../../../../arm-none-eabi/lib/thumb/v7e-m/nofp/libc_nano.a(lib_a-__atexit.o)
 .debug_frame   0x0000000000000000       0x34 /usr/lib/gcc/arm-none-eabi/10.2.0/../../../../arm-none-eabi/lib/thumb/v7e-m/nofp/libc_nano.a(lib_a-__atexit.o)
 .ARM.attributes
                0x0000000000000000       0x2e /usr/lib/gcc/arm-none-eabi/10.2.0/../../../../arm-none-eabi/lib/thumb/v7e-m/nofp/libc_nano.a(lib_a-__atexit.o)
 .text          0x0000000000000000        0x0 /usr/lib/gcc/arm-none-eabi/10.2.0/../../../../arm-none-eabi/lib/thumb/v7e-m/nofp/libc_nano.a(lib_a-__call_atexit.o)
 .data          0x0000000000000000        0x0 /usr/lib/gcc/arm-none-eabi/10.2.0/../../../../arm-none-eabi/lib/thumb/v7e-m/nofp/libc_nano.a(lib_a-__call_atexit.o)
 .bss           0x0000000000000000        0x0 /usr/lib/gcc/arm-none-eabi/10.2.0/../../../../arm-none-eabi/lib/thumb/v7e-m/nofp/libc_nano.a(lib_a-__call_atexit.o)
 .text.__call_exitprocs
                0x0000000000000000       0xbc /usr/lib/gcc/arm-none-eabi/10.2.0/../../../../arm-none-eabi/lib/thumb/v7e-m/nofp/libc_nano.a(lib_a-__call_atexit.o)
 .bss._global_atexit
                0x0000000000000000        0x4 /usr/lib/gcc/arm-none-eabi/10.2.0/../../../../arm-none-eabi/lib/thumb/v7e-m/nofp/libc_nano.a(lib_a-__call_atexit.o)
 .data.__atexit_recursive_mutex
                0x0000000000000000        0x4 /usr/lib/gcc/arm-none-eabi/10.2.0/../../../../arm-none-eabi/lib/thumb/v7e-m/nofp/libc_nano.a(lib_a-__call_atexit.o)
 .debug_frame   0x0000000000000000       0x48 /usr/lib/gcc/arm-none-eabi/10.2.0/../../../../arm-none-eabi/lib/thumb/v7e-m/nofp/libc_nano.a(lib_a-__call_atexit.o)
 .ARM.attributes
                0x0000000000000000       0x2e /usr/lib/gcc/arm-none-eabi/10.2.0/../../../../arm-none-eabi/lib/thumb/v7e-m/nofp/libc_nano.a(lib_a-__call_atexit.o)
 .text          0x0000000000000000        0x0 /usr/lib/gcc/arm-none-eabi/10.2.0/../../../../arm-none-eabi/lib/thumb/v7e-m/nofp/libc_nano.a(lib_a-lock.o)
 .data          0x0000000000000000        0x0 /usr/lib/gcc/arm-none-eabi/10.2.0/../../../../arm-none-eabi/lib/thumb/v7e-m/nofp/libc_nano.a(lib_a-lock.o)
 .bss           0x0000000000000000        0x0 /usr/lib/gcc/arm-none-eabi/10.2.0/../../../../arm-none-eabi/lib/thumb/v7e-m/nofp/libc_nano.a(lib_a-lock.o)
 .text.__retarget_lock_init
                0x0000000000000000        0x2 /usr/lib/gcc/arm-none-eabi/10.2.0/../../../../arm-none-eabi/lib/thumb/v7e-m/nofp/libc_nano.a(lib_a-lock.o)
 .text.__retarget_lock_init_recursive
                0x0000000000000000        0x2 /usr/lib/gcc/arm-none-eabi/10.2.0/../../../../arm-none-eabi/lib/thumb/v7e-m/nofp/libc_nano.a(lib_a-lock.o)
 .text.__retarget_lock_close
                0x0000000000000000        0x2 /usr/lib/gcc/arm-none-eabi/10.2.0/../../../../arm-none-eabi/lib/thumb/v7e-m/nofp/libc_nano.a(lib_a-lock.o)
 .text.__retarget_lock_close_recursive
                0x0000000000000000        0x2 /usr/lib/gcc/arm-none-eabi/10.2.0/../../../../arm-none-eabi/lib/thumb/v7e-m/nofp/libc_nano.a(lib_a-lock.o)
 .text.__retarget_lock_acquire
                0x0000000000000000        0x2 /usr/lib/gcc/arm-none-eabi/10.2.0/../../../../arm-none-eabi/lib/thumb/v7e-m/nofp/libc_nano.a(lib_a-lock.o)
 .text.__retarget_lock_acquire_recursive
                0x0000000000000000        0x2 /usr/lib/gcc/arm-none-eabi/10.2.0/../../../../arm-none-eabi/lib/thumb/v7e-m/nofp/libc_nano.a(lib_a-lock.o)
 .text.__retarget_lock_try_acquire
                0x0000000000000000        0x4 /usr/lib/gcc/arm-none-eabi/10.2.0/../../../../arm-none-eabi/lib/thumb/v7e-m/nofp/libc_nano.a(lib_a-lock.o)
 .text.__retarget_lock_try_acquire_recursive
                0x0000000000000000        0x4 /usr/lib/gcc/arm-none-eabi/10.2.0/../../../../arm-none-eabi/lib/thumb/v7e-m/nofp/libc_nano.a(lib_a-lock.o)
 .text.__retarget_lock_release
                0x0000000000000000        0x2 /usr/lib/gcc/arm-none-eabi/10.2.0/../../../../arm-none-eabi/lib/thumb/v7e-m/nofp/libc_nano.a(lib_a-lock.o)
 .text.__retarget_lock_release_recursive
                0x0000000000000000        0x2 /usr/lib/gcc/arm-none-eabi/10.2.0/../../../../arm-none-eabi/lib/thumb/v7e-m/nofp/libc_nano.a(lib_a-lock.o)
 .debug_frame   0x0000000000000000       0xb0 /usr/lib/gcc/arm-none-eabi/10.2.0/../../../../arm-none-eabi/lib/thumb/v7e-m/nofp/libc_nano.a(lib_a-lock.o)
 .ARM.attributes
                0x0000000000000000       0x2e /usr/lib/gcc/arm-none-eabi/10.2.0/../../../../arm-none-eabi/lib/thumb/v7e-m/nofp/libc_nano.a(lib_a-lock.o)
 COMMON         0x0000000000000000        0x9 /usr/lib/gcc/arm-none-eabi/10.2.0/../../../../arm-none-eabi/lib/thumb/v7e-m/nofp/libc_nano.a(lib_a-lock.o)
 .text          0x0000000000000000        0x0 /usr/lib/gcc/arm-none-eabi/10.2.0/thumb/v7e-m/nofp/crtend.o
 .data          0x0000000000000000        0x0 /usr/lib/gcc/arm-none-eabi/10.2.0/thumb/v7e-m/nofp/crtend.o
 .bss           0x0000000000000000        0x0 /usr/lib/gcc/arm-none-eabi/10.2.0/thumb/v7e-m/nofp/crtend.o
 .eh_frame      0x0000000000000000        0x4 /usr/lib/gcc/arm-none-eabi/10.2.0/thumb/v7e-m/nofp/crtend.o
 .ARM.attributes
                0x0000000000000000       0x2e /usr/lib/gcc/arm-none-eabi/10.2.0/thumb/v7e-m/nofp/crtend.o
 .text          0x0000000000000000        0x0 /usr/lib/gcc/arm-none-eabi/10.2.0/thumb/v7e-m/nofp/crtn.o
 .data          0x0000000000000000        0x0 /usr/lib/gcc/arm-none-eabi/10.2.0/thumb/v7e-m/nofp/crtn.o
 .bss           0x0000000000000000        0x0 /usr/lib/gcc/arm-none-eabi/10.2.0/thumb/v7e-m/nofp/crtn.o

Memory Configuration

Name             Origin             Length             Attributes
rom              0x0000000000000000 0x0000000000100000 xr
ram              0x0000000020000000 0x0000000000040000 xrw
bkupram          0x0000000047000000 0x0000000000002000 xrw
qspi             0x0000000004000000 0x0000000001000000 xrw
*default*        0x0000000000000000 0xffffffffffffffff

Linker script and memory map

LOAD /usr/lib/gcc/arm-none-eabi/10.2.0/thumb/v7e-m/nofp/crti.o
LOAD /usr/lib/gcc/arm-none-eabi/10.2.0/thumb/v7e-m/nofp/crtbegin.o
LOAD /usr/lib/gcc/arm-none-eabi/10.2.0/../../../../arm-none-eabi/lib/thumb/v7e-m/nofp/crt0.o
LOAD ESF/mcu/src/startup_same54.o
LOAD ESF/mcu/src/system_same54.o
LOAD src/main.o
START GROUP
LOAD /usr/lib/gcc/arm-none-eabi/10.2.0/../../../../arm-none-eabi/lib/thumb/v7e-m/nofp/libm.a
END GROUP
START GROUP
LOAD /usr/lib/gcc/arm-none-eabi/10.2.0/thumb/v7e-m/nofp/libgcc.a
LOAD /usr/lib/gcc/arm-none-eabi/10.2.0/../../../../arm-none-eabi/lib/thumb/v7e-m/nofp/libc_nano.a
END GROUP
START GROUP
LOAD /usr/lib/gcc/arm-none-eabi/10.2.0/thumb/v7e-m/nofp/libgcc.a
LOAD /usr/lib/gcc/arm-none-eabi/10.2.0/../../../../arm-none-eabi/lib/thumb/v7e-m/nofp/libc_nano.a
END GROUP
LOAD /usr/lib/gcc/arm-none-eabi/10.2.0/thumb/v7e-m/nofp/crtend.o
LOAD /usr/lib/gcc/arm-none-eabi/10.2.0/thumb/v7e-m/nofp/crtn.o
                0x0000000000010000                STACK_SIZE = DEFINED (STACK_SIZE)?STACK_SIZE:DEFINED (__stack_size__)?__stack_size__:0x10000

.text           0x0000000000000000      0x3d0
                0x0000000000000000                . = ALIGN (0x4)
                0x0000000000000000                _sfixed = .
 *(.vectors .vectors.*)
 .vectors       0x0000000000000000      0x264 ESF/mcu/src/startup_same54.o
                0x0000000000000000                exception_table
 *(.text .text.* .gnu.linkonce.t.*)
 .text.__do_global_dtors_aux
                0x0000000000000264       0x24 /usr/lib/gcc/arm-none-eabi/10.2.0/thumb/v7e-m/nofp/crtbegin.o
 .text.frame_dummy
                0x0000000000000288       0x1c /usr/lib/gcc/arm-none-eabi/10.2.0/thumb/v7e-m/nofp/crtbegin.o
 .text.Dummy_Handler
                0x00000000000002a4        0x2 ESF/mcu/src/startup_same54.o
                0x00000000000002a4                EIC_5_Handler
                0x00000000000002a4                SVCall_Handler
                0x00000000000002a4                SERCOM0_2_Handler
                0x00000000000002a4                EIC_13_Handler
                0x00000000000002a4                EVSYS_0_Handler
                0x00000000000002a4                TCC1_3_Handler
                0x00000000000002a4                DAC_3_Handler
                0x00000000000002a4                TRNG_Handler
                0x00000000000002a4                HardFault_Handler
                0x00000000000002a4                TC2_Handler
                0x00000000000002a4                PDEC_2_Handler
                0x00000000000002a4                EIC_4_Handler
                0x00000000000002a4                AC_Handler
                0x00000000000002a4                SERCOM3_1_Handler
                0x00000000000002a4                SysTick_Handler
                0x00000000000002a4                TCC2_3_Handler
                0x00000000000002a4                SERCOM3_2_Handler
                0x00000000000002a4                PendSV_Handler
                0x00000000000002a4                TC7_Handler
                0x00000000000002a4                ADC1_1_Handler
                0x00000000000002a4                EVSYS_3_Handler
                0x00000000000002a4                PDEC_0_Handler
                0x00000000000002a4                QSPI_Handler
                0x00000000000002a4                NonMaskableInt_Handler
                0x00000000000002a4                TCC0_0_Handler
                0x00000000000002a4                EIC_3_Handler
                0x00000000000002a4                MemManagement_Handler
                0x00000000000002a4                DAC_2_Handler
                0x00000000000002a4                SERCOM0_0_Handler
                0x00000000000002a4                RTC_Handler
                0x00000000000002a4                UsageFault_Handler
                0x00000000000002a4                SERCOM4_0_Handler
                0x00000000000002a4                EIC_10_Handler
                0x00000000000002a4                SERCOM0_3_Handler
                0x00000000000002a4                EIC_11_Handler
                0x00000000000002a4                EIC_9_Handler
                0x00000000000002a4                OSC32KCTRL_Handler
                0x00000000000002a4                TCC2_1_Handler
                0x00000000000002a4                SUPC_1_Handler
                0x00000000000002a4                TCC0_5_Handler
                0x00000000000002a4                TCC0_6_Handler
                0x00000000000002a4                SERCOM6_2_Handler
                0x00000000000002a4                EVSYS_1_Handler
                0x00000000000002a4                TCC1_4_Handler
                0x00000000000002a4                TC6_Handler
                0x00000000000002a4                DMAC_0_Handler
                0x00000000000002a4                WDT_Handler
                0x00000000000002a4                CAN0_Handler
                0x00000000000002a4                EIC_8_Handler
                0x00000000000002a4                EIC_15_Handler
                0x00000000000002a4                SERCOM6_0_Handler
                0x00000000000002a4                SERCOM5_0_Handler
                0x00000000000002a4                TC4_Handler
                0x00000000000002a4                TC1_Handler
                0x00000000000002a4                OSCCTRL_4_Handler
                0x00000000000002a4                SERCOM4_3_Handler
                0x00000000000002a4                EIC_12_Handler
                0x00000000000002a4                DMAC_4_Handler
                0x00000000000002a4                TCC4_2_Handler
                0x00000000000002a4                PAC_Handler
                0x00000000000002a4                TCC1_0_Handler
                0x00000000000002a4                USB_0_Handler
                0x00000000000002a4                OSCCTRL_0_Handler
                0x00000000000002a4                EIC_0_Handler
                0x00000000000002a4                OSCCTRL_3_Handler
                0x00000000000002a4                SERCOM4_1_Handler
                0x00000000000002a4                TC3_Handler
                0x00000000000002a4                Dummy_Handler
                0x00000000000002a4                TCC3_0_Handler
                0x00000000000002a4                TCC2_2_Handler
                0x00000000000002a4                SERCOM5_1_Handler
                0x00000000000002a4                TCC1_1_Handler
                0x00000000000002a4                DMAC_2_Handler
                0x00000000000002a4                ADC0_0_Handler
                0x00000000000002a4                SERCOM0_1_Handler
                0x00000000000002a4                OSCCTRL_2_Handler
                0x00000000000002a4                ADC1_0_Handler
                0x00000000000002a4                TCC1_2_Handler
                0x00000000000002a4                SERCOM7_1_Handler
                0x00000000000002a4                USB_1_Handler
                0x00000000000002a4                PM_Handler
                0x00000000000002a4                SERCOM6_3_Handler
                0x00000000000002a4                SERCOM2_3_Handler
                0x00000000000002a4                DAC_4_Handler
                0x00000000000002a4                TCC3_2_Handler
                0x00000000000002a4                SERCOM7_0_Handler
                0x00000000000002a4                TCC0_2_Handler
                0x00000000000002a4                DMAC_1_Handler
                0x00000000000002a4                TCC4_0_Handler
                0x00000000000002a4                SERCOM7_3_Handler
                0x00000000000002a4                GMAC_Handler
                0x00000000000002a4                SDHC1_Handler
                0x00000000000002a4                USB_3_Handler
                0x00000000000002a4                SERCOM7_2_Handler
                0x00000000000002a4                CAN1_Handler
                0x00000000000002a4                TCC2_0_Handler
                0x00000000000002a4                PDEC_1_Handler
                0x00000000000002a4                TCC4_1_Handler
                0x00000000000002a4                SERCOM5_3_Handler
                0x00000000000002a4                USB_2_Handler
                0x00000000000002a4                SERCOM6_1_Handler
                0x00000000000002a4                SDHC0_Handler
                0x00000000000002a4                SERCOM1_1_Handler
                0x00000000000002a4                I2S_Handler
                0x00000000000002a4                EIC_2_Handler
                0x00000000000002a4                PCC_Handler
                0x00000000000002a4                DAC_0_Handler
                0x00000000000002a4                TCC0_1_Handler
                0x00000000000002a4                SERCOM1_3_Handler
                0x00000000000002a4                EIC_6_Handler
                0x00000000000002a4                OSCCTRL_1_Handler
                0x00000000000002a4                SERCOM1_0_Handler
                0x00000000000002a4                PUKCC_Handler
                0x00000000000002a4                SERCOM2_1_Handler
                0x00000000000002a4                SERCOM1_2_Handler
                0x00000000000002a4                SERCOM3_0_Handler
                0x00000000000002a4                EIC_1_Handler
                0x00000000000002a4                SERCOM4_2_Handler
                0x00000000000002a4                EVSYS_4_Handler
                0x00000000000002a4                EIC_7_Handler
                0x00000000000002a4                NVMCTRL_1_Handler
                0x00000000000002a4                SERCOM5_2_Handler
                0x00000000000002a4                SERCOM3_3_Handler
                0x00000000000002a4                ADC0_1_Handler
                0x00000000000002a4                SERCOM2_2_Handler
                0x00000000000002a4                TCC3_1_Handler
                0x00000000000002a4                EIC_14_Handler
                0x00000000000002a4                DAC_1_Handler
                0x00000000000002a4                NVMCTRL_0_Handler
                0x00000000000002a4                MCLK_Handler
                0x00000000000002a4                EVSYS_2_Handler
                0x00000000000002a4                SUPC_0_Handler
                0x00000000000002a4                BusFault_Handler
                0x00000000000002a4                FREQM_Handler
                0x00000000000002a4                TC0_Handler
                0x00000000000002a4                TCC0_3_Handler
                0x00000000000002a4                DMAC_3_Handler
                0x00000000000002a4                DebugMonitor_Handler
                0x00000000000002a4                TCC0_4_Handler
                0x00000000000002a4                RAMECC_Handler
                0x00000000000002a4                TC5_Handler
                0x00000000000002a4                SERCOM2_0_Handler
                0x00000000000002a4                AES_Handler
                0x00000000000002a4                ICM_Handler
 *fill*         0x00000000000002a6        0x2 
 .text.Reset_Handler
                0x00000000000002a8       0x90 ESF/mcu/src/startup_same54.o
                0x00000000000002a8                Reset_Handler
 .text.startup.main
                0x0000000000000338        0x4 src/main.o
                0x0000000000000338                main
 .text.__libc_init_array
                0x000000000000033c       0x48 /usr/lib/gcc/arm-none-eabi/10.2.0/../../../../arm-none-eabi/lib/thumb/v7e-m/nofp/libc_nano.a(lib_a-init.o)
                0x000000000000033c                __libc_init_array
 .text.memcpy   0x0000000000000384       0x1c /usr/lib/gcc/arm-none-eabi/10.2.0/../../../../arm-none-eabi/lib/thumb/v7e-m/nofp/libc_nano.a(lib_a-memcpy-stub.o)
                0x0000000000000384                memcpy
 .text.memset   0x00000000000003a0       0x10 /usr/lib/gcc/arm-none-eabi/10.2.0/../../../../arm-none-eabi/lib/thumb/v7e-m/nofp/libc_nano.a(lib_a-memset.o)
                0x00000000000003a0                memset
 *(.glue_7t)
 .glue_7t       0x00000000000003b0        0x0 linker stubs
 *(.glue_7)
 .glue_7        0x00000000000003b0        0x0 linker stubs
 *(.rodata .rodata* .gnu.linkonce.r.*)
 *(.ARM.extab* .gnu.linkonce.armextab.*)
                0x00000000000003b0                . = ALIGN (0x4)
 *(.init)
 .init          0x00000000000003b0        0x4 /usr/lib/gcc/arm-none-eabi/10.2.0/thumb/v7e-m/nofp/crti.o
                0x00000000000003b0                _init
 .init          0x00000000000003b4        0x8 /usr/lib/gcc/arm-none-eabi/10.2.0/thumb/v7e-m/nofp/crtn.o
                0x00000000000003bc                . = ALIGN (0x4)
                0x00000000000003bc                __preinit_array_start = .
 *(.preinit_array)
                0x00000000000003bc                __preinit_array_end = .
                0x00000000000003bc                . = ALIGN (0x4)
                0x00000000000003bc                __init_array_start = .
 *(SORT_BY_NAME(.init_array.*))
 *(.init_array)
 .init_array    0x00000000000003bc        0x4 /usr/lib/gcc/arm-none-eabi/10.2.0/thumb/v7e-m/nofp/crtbegin.o
                0x00000000000003c0                __init_array_end = .
                0x00000000000003c0                . = ALIGN (0x4)
 *crtbegin.o(.ctors)
 *(EXCLUDE_FILE(*crtend.o) .ctors)
 *(SORT_BY_NAME(.ctors.*))
 *crtend.o(.ctors)
                0x00000000000003c0                . = ALIGN (0x4)
 *(.fini)
 .fini          0x00000000000003c0        0x4 /usr/lib/gcc/arm-none-eabi/10.2.0/thumb/v7e-m/nofp/crti.o
                0x00000000000003c0                _fini
 .fini          0x00000000000003c4        0x8 /usr/lib/gcc/arm-none-eabi/10.2.0/thumb/v7e-m/nofp/crtn.o
                0x00000000000003cc                . = ALIGN (0x4)
                0x00000000000003cc                __fini_array_start = .
 *(.fini_array)
 .fini_array    0x00000000000003cc        0x4 /usr/lib/gcc/arm-none-eabi/10.2.0/thumb/v7e-m/nofp/crtbegin.o
 *(SORT_BY_NAME(.fini_array.*))
                0x00000000000003d0                __fini_array_end = .
 *crtbegin.o(.dtors)
 *(EXCLUDE_FILE(*crtend.o) .dtors)
 *(SORT_BY_NAME(.dtors.*))
 *crtend.o(.dtors)
                0x00000000000003d0                . = ALIGN (0x4)
                0x00000000000003d0                _efixed = .
                [!provide]                        PROVIDE (__exidx_start = .)

.vfp11_veneer   0x00000000000003d0        0x0
 .vfp11_veneer  0x00000000000003d0        0x0 linker stubs

.v4_bx          0x00000000000003d0        0x0
 .v4_bx         0x00000000000003d0        0x0 linker stubs

.iplt           0x00000000000003d0        0x0
 .iplt          0x00000000000003d0        0x0 /usr/lib/gcc/arm-none-eabi/10.2.0/thumb/v7e-m/nofp/crtbegin.o

.igot.plt       0x00000000000003d0        0x0
 .igot.plt      0x00000000000003d0        0x0 /usr/lib/gcc/arm-none-eabi/10.2.0/thumb/v7e-m/nofp/crtbegin.o

.eh_frame       0x00000000000003d0        0x0
 .eh_frame      0x00000000000003d0        0x0 /usr/lib/gcc/arm-none-eabi/10.2.0/thumb/v7e-m/nofp/crtbegin.o

.rel.dyn        0x00000000000003d0        0x0
 .rel.iplt      0x00000000000003d0        0x0 /usr/lib/gcc/arm-none-eabi/10.2.0/thumb/v7e-m/nofp/crtbegin.o

.ARM.exidx
 *(.ARM.exidx* .gnu.linkonce.armexidx.*)
                [!provide]                        PROVIDE (__exidx_end = .)
                0x00000000000003d0                . = ALIGN (0x4)
                0x00000000000003d0                _etext = .

.relocate       0x0000000020000000        0x0 load address 0x00000000000003d0
                0x0000000020000000                . = ALIGN (0x4)
                0x0000000020000000                _srelocate = .
 *(.ramfunc .ramfunc.*)
 *(.data .data.*)
                0x0000000020000000                . = ALIGN (0x4)
                0x0000000020000000                _erelocate = .

.bkupram        0x0000000047000000        0x0
                0x0000000047000000                . = ALIGN (0x8)
                0x0000000047000000                _sbkupram = .
 *(.bkupram .bkupram.*)
                0x0000000047000000                . = ALIGN (0x8)
                0x0000000047000000                _ebkupram = .

.qspi           0x0000000004000000        0x0
                0x0000000004000000                . = ALIGN (0x8)
                0x0000000004000000                _sqspi = .
 *(.qspi .qspi.*)
                0x0000000004000000                . = ALIGN (0x8)
                0x0000000004000000                _eqspi = .

.bss            0x0000000020000000       0x1c
                0x0000000020000000                . = ALIGN (0x4)
                0x0000000020000000                _sbss = .
                0x0000000020000000                _szero = .
 *(.bss .bss.*)
 .bss.completed.1
                0x0000000020000000        0x1 /usr/lib/gcc/arm-none-eabi/10.2.0/thumb/v7e-m/nofp/crtbegin.o
 *fill*         0x0000000020000001        0x3 
 .bss.object.0  0x0000000020000004       0x18 /usr/lib/gcc/arm-none-eabi/10.2.0/thumb/v7e-m/nofp/crtbegin.o
 *(COMMON)
                0x000000002000001c                . = ALIGN (0x4)
                0x000000002000001c                _ebss = .
                0x000000002000001c                _ezero = .

.stack          0x000000002000001c    0x10004
                0x0000000020000020                . = ALIGN (0x8)
 *fill*         0x000000002000001c        0x4 
                0x0000000020000020                _sstack = .
                0x0000000020010020                . = (. + STACK_SIZE)
 *fill*         0x0000000020000020    0x10000 
                0x0000000020010020                . = ALIGN (0x8)
                0x0000000020010020                _estack = .
                0x0000000020010020                . = ALIGN (0x4)
                0x0000000020010020                _end = .
OUTPUT(e54testdir.elf elf32-littlearm)
LOAD linker stubs

.ARM.attributes
                0x0000000000000000       0x2e
 .ARM.attributes
                0x0000000000000000       0x1e /usr/lib/gcc/arm-none-eabi/10.2.0/thumb/v7e-m/nofp/crti.o
 .ARM.attributes
                0x000000000000001e       0x2e /usr/lib/gcc/arm-none-eabi/10.2.0/thumb/v7e-m/nofp/crtbegin.o
 .ARM.attributes
                0x000000000000004c       0x32 ESF/mcu/src/startup_same54.o
 .ARM.attributes
                0x000000000000007e       0x32 src/main.o
 .ARM.attributes
                0x00000000000000b0       0x2e /usr/lib/gcc/arm-none-eabi/10.2.0/../../../../arm-none-eabi/lib/thumb/v7e-m/nofp/libc_nano.a(lib_a-init.o)
 .ARM.attributes
                0x00000000000000de       0x2e /usr/lib/gcc/arm-none-eabi/10.2.0/../../../../arm-none-eabi/lib/thumb/v7e-m/nofp/libc_nano.a(lib_a-memcpy-stub.o)
 .ARM.attributes
                0x000000000000010c       0x2e /usr/lib/gcc/arm-none-eabi/10.2.0/../../../../arm-none-eabi/lib/thumb/v7e-m/nofp/libc_nano.a(lib_a-memset.o)
 .ARM.attributes
                0x000000000000013a       0x1e /usr/lib/gcc/arm-none-eabi/10.2.0/thumb/v7e-m/nofp/crtn.o

.comment        0x0000000000000000       0x1e
 .comment       0x0000000000000000       0x1e ESF/mcu/src/startup_same54.o
                                         0x1f (size before relaxing)
 .comment       0x000000000000001e       0x1f src/main.o

.debug_info     0x0000000000000000      0xd0a
 .debug_info    0x0000000000000000      0xc84 ESF/mcu/src/startup_same54.o
 .debug_info    0x0000000000000c84       0x86 src/main.o

.debug_abbrev   0x0000000000000000      0x200
 .debug_abbrev  0x0000000000000000      0x1b9 ESF/mcu/src/startup_same54.o
 .debug_abbrev  0x00000000000001b9       0x47 src/main.o

.debug_aranges  0x0000000000000000       0x48
 .debug_aranges
                0x0000000000000000       0x28 ESF/mcu/src/startup_same54.o
 .debug_aranges
                0x0000000000000028       0x20 src/main.o

.debug_ranges   0x0000000000000000       0x28
 .debug_ranges  0x0000000000000000       0x18 ESF/mcu/src/startup_same54.o
 .debug_ranges  0x0000000000000018       0x10 src/main.o

.debug_macro    0x0000000000000000    0x26037
 .debug_macro   0x0000000000000000      0x4b2 ESF/mcu/src/startup_same54.o
 .debug_macro   0x00000000000004b2      0xa78 ESF/mcu/src/startup_same54.o
 .debug_macro   0x0000000000000f2a       0x22 ESF/mcu/src/startup_same54.o
 .debug_macro   0x0000000000000f4c       0x8e ESF/mcu/src/startup_same54.o
 .debug_macro   0x0000000000000fda       0x51 ESF/mcu/src/startup_same54.o
 .debug_macro   0x000000000000102b      0x103 ESF/mcu/src/startup_same54.o
 .debug_macro   0x000000000000112e       0x6a ESF/mcu/src/startup_same54.o
 .debug_macro   0x0000000000001198      0x1df ESF/mcu/src/startup_same54.o
 .debug_macro   0x0000000000001377       0x4e ESF/mcu/src/startup_same54.o
 .debug_macro   0x00000000000013c5       0x1c ESF/mcu/src/startup_same54.o
 .debug_macro   0x00000000000013e1       0x22 ESF/mcu/src/startup_same54.o
 .debug_macro   0x0000000000001403       0xd9 ESF/mcu/src/startup_same54.o
 .debug_macro   0x00000000000014dc     0x102d ESF/mcu/src/startup_same54.o
 .debug_macro   0x0000000000002509      0x11f ESF/mcu/src/startup_same54.o
 .debug_macro   0x0000000000002628      0x706 ESF/mcu/src/startup_same54.o
 .debug_macro   0x0000000000002d2e      0xb5b ESF/mcu/src/startup_same54.o
 .debug_macro   0x0000000000003889      0x3c0 ESF/mcu/src/startup_same54.o
 .debug_macro   0x0000000000003c49     0x2d61 ESF/mcu/src/startup_same54.o
 .debug_macro   0x00000000000069aa      0x336 ESF/mcu/src/startup_same54.o
 .debug_macro   0x0000000000006ce0      0x3b7 ESF/mcu/src/startup_same54.o
 .debug_macro   0x0000000000007097      0x668 ESF/mcu/src/startup_same54.o
 .debug_macro   0x00000000000076ff     0x143f ESF/mcu/src/startup_same54.o
 .debug_macro   0x0000000000008b3e      0x651 ESF/mcu/src/startup_same54.o
 .debug_macro   0x000000000000918f      0x67b ESF/mcu/src/startup_same54.o
 .debug_macro   0x000000000000980a      0x6d7 ESF/mcu/src/startup_same54.o
 .debug_macro   0x0000000000009ee1      0x172 ESF/mcu/src/startup_same54.o
 .debug_macro   0x000000000000a053      0x395 ESF/mcu/src/startup_same54.o
 .debug_macro   0x000000000000a3e8     0x19dd ESF/mcu/src/startup_same54.o
 .debug_macro   0x000000000000bdc5       0x3a ESF/mcu/src/startup_same54.o
 .debug_macro   0x000000000000bdff      0x72a ESF/mcu/src/startup_same54.o
 .debug_macro   0x000000000000c529      0xb12 ESF/mcu/src/startup_same54.o
 .debug_macro   0x000000000000d03b      0x5d7 ESF/mcu/src/startup_same54.o
 .debug_macro   0x000000000000d612      0xbc0 ESF/mcu/src/startup_same54.o
 .debug_macro   0x000000000000e1d2      0x9b9 ESF/mcu/src/startup_same54.o
 .debug_macro   0x000000000000eb8b      0x2a3 ESF/mcu/src/startup_same54.o
 .debug_macro   0x000000000000ee2e      0x8cb ESF/mcu/src/startup_same54.o
 .debug_macro   0x000000000000f6f9      0x1ea ESF/mcu/src/startup_same54.o
 .debug_macro   0x000000000000f8e3      0x8f4 ESF/mcu/src/startup_same54.o
 .debug_macro   0x00000000000101d7      0x216 ESF/mcu/src/startup_same54.o
 .debug_macro   0x00000000000103ed      0x3f9 ESF/mcu/src/startup_same54.o
 .debug_macro   0x00000000000107e6      0x620 ESF/mcu/src/startup_same54.o
 .debug_macro   0x0000000000010e06      0x10d ESF/mcu/src/startup_same54.o
 .debug_macro   0x0000000000010f13       0xb8 ESF/mcu/src/startup_same54.o
 .debug_macro   0x0000000000010fcb     0x1df7 ESF/mcu/src/startup_same54.o
 .debug_macro   0x0000000000012dc2     0x2e69 ESF/mcu/src/startup_same54.o
 .debug_macro   0x0000000000015c2b     0x11ed ESF/mcu/src/startup_same54.o
 .debug_macro   0x0000000000016e18      0x50e ESF/mcu/src/startup_same54.o
 .debug_macro   0x0000000000017326      0x930 ESF/mcu/src/startup_same54.o
 .debug_macro   0x0000000000017c56     0x1ad8 ESF/mcu/src/startup_same54.o
 .debug_macro   0x000000000001972e       0xe7 ESF/mcu/src/startup_same54.o
 .debug_macro   0x0000000000019815     0x13e6 ESF/mcu/src/startup_same54.o
 .debug_macro   0x000000000001abfb      0x36a ESF/mcu/src/startup_same54.o
 .debug_macro   0x000000000001af65       0x94 ESF/mcu/src/startup_same54.o
 .debug_macro   0x000000000001aff9       0xdc ESF/mcu/src/startup_same54.o
 .debug_macro   0x000000000001b0d5       0xe2 ESF/mcu/src/startup_same54.o
 .debug_macro   0x000000000001b1b7       0xdc ESF/mcu/src/startup_same54.o
 .debug_macro   0x000000000001b293      0x149 ESF/mcu/src/startup_same54.o
 .debug_macro   0x000000000001b3dc      0x149 ESF/mcu/src/startup_same54.o
 .debug_macro   0x000000000001b525       0x46 ESF/mcu/src/startup_same54.o
 .debug_macro   0x000000000001b56b       0x4c ESF/mcu/src/startup_same54.o
 .debug_macro   0x000000000001b5b7       0xc4 ESF/mcu/src/startup_same54.o
 .debug_macro   0x000000000001b67b      0x7d5 ESF/mcu/src/startup_same54.o
 .debug_macro   0x000000000001be50       0xb8 ESF/mcu/src/startup_same54.o
 .debug_macro   0x000000000001bf08       0x7c ESF/mcu/src/startup_same54.o
 .debug_macro   0x000000000001bf84      0xc20 ESF/mcu/src/startup_same54.o
 .debug_macro   0x000000000001cba4       0x46 ESF/mcu/src/startup_same54.o
 .debug_macro   0x000000000001cbea      0x25b ESF/mcu/src/startup_same54.o
 .debug_macro   0x000000000001ce45      0x31a ESF/mcu/src/startup_same54.o
 .debug_macro   0x000000000001d15f      0x170 ESF/mcu/src/startup_same54.o
 .debug_macro   0x000000000001d2cf       0x7c ESF/mcu/src/startup_same54.o
 .debug_macro   0x000000000001d34b       0xbe ESF/mcu/src/startup_same54.o
 .debug_macro   0x000000000001d409       0x4c ESF/mcu/src/startup_same54.o
 .debug_macro   0x000000000001d455       0x82 ESF/mcu/src/startup_same54.o
 .debug_macro   0x000000000001d4d7      0x1a3 ESF/mcu/src/startup_same54.o
 .debug_macro   0x000000000001d67a       0x46 ESF/mcu/src/startup_same54.o
 .debug_macro   0x000000000001d6c0       0x6a ESF/mcu/src/startup_same54.o
 .debug_macro   0x000000000001d72a       0x46 ESF/mcu/src/startup_same54.o
 .debug_macro   0x000000000001d770       0x88 ESF/mcu/src/startup_same54.o
 .debug_macro   0x000000000001d7f8       0x46 ESF/mcu/src/startup_same54.o
 .debug_macro   0x000000000001d83e      0x24e ESF/mcu/src/startup_same54.o
 .debug_macro   0x000000000001da8c       0x1c ESF/mcu/src/startup_same54.o
 .debug_macro   0x000000000001daa8       0x76 ESF/mcu/src/startup_same54.o
 .debug_macro   0x000000000001db1e       0x3a ESF/mcu/src/startup_same54.o
 .debug_macro   0x000000000001db58       0x2e ESF/mcu/src/startup_same54.o
 .debug_macro   0x000000000001db86      0x196 ESF/mcu/src/startup_same54.o
 .debug_macro   0x000000000001dd1c      0x16f ESF/mcu/src/startup_same54.o
 .debug_macro   0x000000000001de8b      0x16f ESF/mcu/src/startup_same54.o
 .debug_macro   0x000000000001dffa      0x25d ESF/mcu/src/startup_same54.o
 .debug_macro   0x000000000001e257      0x25d ESF/mcu/src/startup_same54.o
 .debug_macro   0x000000000001e4b4      0x25d ESF/mcu/src/startup_same54.o
 .debug_macro   0x000000000001e711      0x25d ESF/mcu/src/startup_same54.o
 .debug_macro   0x000000000001e96e      0x25d ESF/mcu/src/startup_same54.o
 .debug_macro   0x000000000001ebcb      0x25d ESF/mcu/src/startup_same54.o
 .debug_macro   0x000000000001ee28      0x25d ESF/mcu/src/startup_same54.o
 .debug_macro   0x000000000001f085      0x25d ESF/mcu/src/startup_same54.o
 .debug_macro   0x000000000001f2e2       0x52 ESF/mcu/src/startup_same54.o
 .debug_macro   0x000000000001f334       0xfa ESF/mcu/src/startup_same54.o
 .debug_macro   0x000000000001f42e       0xfa ESF/mcu/src/startup_same54.o
 .debug_macro   0x000000000001f528       0xfa ESF/mcu/src/startup_same54.o
 .debug_macro   0x000000000001f622       0xfa ESF/mcu/src/startup_same54.o
 .debug_macro   0x000000000001f71c       0xfa ESF/mcu/src/startup_same54.o
 .debug_macro   0x000000000001f816       0xfa ESF/mcu/src/startup_same54.o
 .debug_macro   0x000000000001f910       0xfa ESF/mcu/src/startup_same54.o
 .debug_macro   0x000000000001fa0a       0xfa ESF/mcu/src/startup_same54.o
 .debug_macro   0x000000000001fb04      0x148 ESF/mcu/src/startup_same54.o
 .debug_macro   0x000000000001fc4c      0x124 ESF/mcu/src/startup_same54.o
 .debug_macro   0x000000000001fd70      0x106 ESF/mcu/src/startup_same54.o
 .debug_macro   0x000000000001fe76       0xee ESF/mcu/src/startup_same54.o
 .debug_macro   0x000000000001ff64       0xee ESF/mcu/src/startup_same54.o
 .debug_macro   0x0000000000020052       0x2e ESF/mcu/src/startup_same54.o
 .debug_macro   0x0000000000020080      0x46a ESF/mcu/src/startup_same54.o
 .debug_macro   0x00000000000204ea       0x3a ESF/mcu/src/startup_same54.o
 .debug_macro   0x0000000000020524      0x59f ESF/mcu/src/startup_same54.o
 .debug_macro   0x0000000000020ac3     0x4ff3 ESF/mcu/src/startup_same54.o
 .debug_macro   0x0000000000025ab6       0xcf ESF/mcu/src/startup_same54.o
 .debug_macro   0x0000000000025b85      0x4b2 src/main.o

.debug_line     0x0000000000000000      0xcd8
 .debug_line    0x0000000000000000      0x6b9 ESF/mcu/src/startup_same54.o
 .debug_line    0x00000000000006b9      0x61f src/main.o

.debug_str      0x0000000000000000    0xf108b
 .debug_str     0x0000000000000000    0xf107d ESF/mcu/src/startup_same54.o
                                      0xf1467 (size before relaxing)
 .debug_str     0x00000000000f107d        0xe src/main.o
                                      0xf0820 (size before relaxing)

.debug_frame    0x0000000000000000       0xcc
 .debug_frame   0x0000000000000000       0x38 ESF/mcu/src/startup_same54.o
 .debug_frame   0x0000000000000038       0x20 src/main.o
 .debug_frame   0x0000000000000058       0x2c /usr/lib/gcc/arm-none-eabi/10.2.0/../../../../arm-none-eabi/lib/thumb/v7e-m/nofp/libc_nano.a(lib_a-init.o)
 .debug_frame   0x0000000000000084       0x28 /usr/lib/gcc/arm-none-eabi/10.2.0/../../../../arm-none-eabi/lib/thumb/v7e-m/nofp/libc_nano.a(lib_a-memcpy-stub.o)
 .debug_frame   0x00000000000000ac       0x20 /usr/lib/gcc/arm-none-eabi/10.2.0/../../../../arm-none-eabi/lib/thumb/v7e-m/nofp/libc_nano.a(lib_a-memset.o)
